:020000040000FA
:04000000CCEF03F04E
:0400080065EF27F089
:08001800CCEF27F00F0B436E43
:10002000000EF76E3A0EF66E4350F626D8B0F72A59
:10003000F29E0900F28EF550120030313233343521
:100040003637383941424344454681C218F019D801
:100050002DC083F22EC084F22FC085F230C086F20C
:1000600031C087F2120082C218F00BD82DC088F27E
:100070002EC089F22FC08AF230C08BF231C08CF2D0
:100080001200AEEC32F02DEC34F06DEC36F000ECFA
:1000900035F06DEC36F0C3EC34F080EC30F0E4EC8D
:1000A0003BF06AEC30F054EC30F0C3EF34F020C297
:1000B00018F0D88018AED89012003EC218F0D88040
:1000C00018AED89012002BC22DF02CC22EF02DC2EB
:1000D0002FF02EC230F02FC231F0ECEC3BF02DC0EF
:1000E00030F22EC031F22FC032F230C033F231C0C4
:1000F00034F212001CC22DF01DC22EF01EC22FF0D1
:100100001FC230F020C231F026C232F027C233F0D5
:1001100028C234F029C235F02AC236F000EC35F09E
:100120002DC02BF22EC02CF22FC02DF230C02EF29B
:1001300031C02FF231AE0CD0C9EC36F032C02BF208
:1001400033C02CF234C02DF235C02EF236C02FF25F
:100150001200A7EC32F02DEC34F008C232F009C2E4
:1001600033F00AC234F00BC235F00CC236F043EC67
:1001700034F00DC232F00EC233F00FC234F010C2B0
:1001800035F011C236F006EC35F05DC232F05EC2D9
:1001900033F05FC234F060C235F061C236F006EF72
:1001A00035F072C018F073C019F0D3DF2DC03AF2E9
:1001B0002EC03BF22FC03CF230C03DF231C03EF2C7
:1001C000120078C018F079C019F0C3DF2DC053F2C7
:1001D0002EC054F22FC055F230C056F231C057F243
:1001E00012006CC018F06DC019F0B3DF2DC021F201
:1001F0002EC022F22FC023F230C024F231C025F2EB
:1002000012006FC018F070C019F0A3DF2DC035F2D6
:100210002EC036F22FC037F230C038F231C039F27A
:10022000120076C018F077C019F093DF2DC04EF29F
:100230002EC04FF22FC050F230C051F231C052F2F6
:10024000120062C018F063C019F083DF2DC01CF2E9
:100250002EC01DF22FC01EF230C01FF231C020F29E
:100260001200A7EC32F02DEC34F012C232F013C2BF
:1002700033F014C234F015C235F016C236F043EC38
:1002800034F017C232F018C233F019C234F01AC277
:1002900035F01BC236F006EC35F05DC232F05EC2BE
:1002A00033F05FC234F060C235F061C236F006EF61
:1002B00035F074C018F075C019F0D3DF2DC03FF2CF
:1002C0002EC040F22FC041F230C042F231C043F2A2
:1002D00012007AC018F07BC019F0C3DF2DC058F2AD
:1002E0002EC059F22FC05AF230C05BF231C05CF21E
:1002F000120067C018F068C019F0B3DF2DC026F2F5
:100300002EC027F22FC028F230C029F231C02AF2C5
:1003100012007C6B7E6B7F6B816B1200140E7C6510
:1003200002D0140E7C6F7C517D5DD8B403D07CC0AC
:100330007DF03D867E517C5DD8A00AD003C282F05C
:100340007E517C5DD8B404D07CC07EF03D8613D055
:10035000826711D03DB80DD083670DD03FBA03D06E
:100360000A0E836F02D00A0E836F3D867E677E077A
:1003700002D07E6B3D861200140E7F6502D0140EF3
:100380007F6F7F51805DD8B403D07FC080F03D8601
:1003900081517F5DD8A00AD003C284F081517F5D76
:1003A000D8B404D07FC081F03D860ED084670CD0D5
:1003B0003DBA08D0856708D00A0E856F3D868167F3
:1003C000810702D0816B3D861200400E506E656B36
:1003D000666B186A66EC25F0545065275550662305
:1003E000502EF8D7D890663365331836D8906633D8
:1003F00065331836D890663365331836030E1864A3
:1004000003D0652BD8B4662B1200400E506E606B83
:10041000616B186A68EC25F05450602755506123D1
:10042000502EF8D7D890613360331836D8906133A6
:1004300060331836D890613360331836030E186471
:1004400003D0602BD8B4612B1200080E506E606B85
:10045000616B656B666B6A6B6B6B68EC25F0545077
:1004600060275550612366EC25F0545065275550A0
:1004700066236AEC25F054506A2755506B23502EA2
:10048000ECD71200420E366E4C0E356E990E346E5D
:10049000990E336E9A0E326E0AD0410E366ECC0E25
:1004A000356E990E346E990E336E9A0E326E43ECA1
:1004B00034F0D3EC31F012AE02D00E6A0F6A41EC88
:1004C00030F0FF0E186E030E196E0F50195C02E12A
:1004D0000E50185CD8B004D018C00EF019C00FF040
:1004E0001200420E316E200E306E2D6A2E6A2F6A77
:1004F0002BC232F02CC233F02DC234F02EC235F0B4
:100500002FC236F000EC35F0C8DF0EC097F00FC0F8
:1005100098F012002BC22DF02CC22EF02DC22FF01D
:100520002EC230F02FC231F0B8DF0EC097F00FC0EE
:1005300098F0120030C22DF031C22EF032C22FF0EE
:1005400033C230F034C231F05EEC36F000EC35F0FE
:1005500088C232F089C233F08AC234F08BC235F0DF
:100560008CC236F043EC34F08DDF0EC097F00FC034
:1005700098F0120026C22DF027C22EF028C22FF0CC
:1005800029C230F02AC231F062C232F063C233F0C5
:1005900064C234F065C235F066C236F000EC35F066
:1005A00071DF0EC097F00FC098F0120026C22DF038
:1005B00027C22EF028C22FF029C230F02AC231F013
:1005C0006DEC36F006EC35F0DFD726C22DF027C2F1
:1005D0002EF028C22FF029C230F02AC231F0E4EC0C
:1005E0003BF006EC35F0D0D74EC22DF04FC22EF0C6
:1005F00050C22FF051C230F052C231F015D80EC0A7
:1006000091F00FC092F0120053C22DF054C22EF0A0
:1006100055C22FF056C230F057C231F005D80EC087
:1006200093F00FC094F0120062C232F063C233F054
:1006300064C234F065C235F066C236F000EC35F0C5
:1006400021DF120030C22DF031C22EF032C22FF065
:1006500033C230F034C231F05EEC36F000EC35F0ED
:1006600083C232F084C233F085C234F086C235F0E2
:1006700087C236F043EC34F07DD80EC07FF0120014
:100680000CD8140E7F6502D0140E7F6F140E186EF6
:100690007F51185E18C07FF012002BC22DF02CC2C3
:1006A0002EF02DC22FF02EC230F02FC231F066ECAA
:1006B00036F0C3EC34F05ED80EC07FF0120026C2D4
:1006C0002DF027C22EF028C22FF029C230F02AC206
:1006D00031F0E4EC3BF006EC35F019D026C22DF0F9
:1006E00027C22EF028C22FF029C230F02AC231F0E2
:1006F0006DEC36F006EC35F00AD026C22DF027C29C
:100700002EF028C22FF029C230F02AC231F062C286
:1007100032F063C233F064C234F065C235F066C2B1
:1007200036F026D80EC07FF0120021C22DF022C272
:100730002EF023C22FF024C230F025C231F00AD0AF
:100740001CC22DF01DC22EF01EC22FF01FC230F0B1
:1007500020C231F062C232F063C233F064C234F0BE
:1007600065C235F066C236F003D80EC07CF01200C8
:1007700000EC35F0D3EC31F012BE0E6A1200000E20
:10078000A7EC21F095EC3AF074EC39F052EC20F043
:1007900052EC20F052EF20F061EC22F0D0B622D0E3
:1007A000B42B9FEC21F0000EF86E5D0EF76E5C0E20
:1007B000F66EB9EC21F0000EF86E5D0EF76E9E0E2F
:1007C000F66EB9EC21F041EC30F0B4C018F095ECC5
:1007D0003AF074EC39F052EC20F09FEC21F03D86B9
:1007E0003D8226D03BEC22F0C0EC22F070EC20F0F1
:1007F0008EEC20F0C2EC21F0B2EC20F0E2EC21F023
:10080000B0EC22F0C4EC22F09FEC21F0DDEC22F001
:100810003D86908999693D82626B636B646B6C6BFA
:100820006D6B6E6B676B686B696B3F963F943F981F
:10083000040059523BE03DAC5EEC36F03DBCBEECF2
:1008400036F062C22DF063C22EF064C22FF065C292
:1008500030F066C231F059BE03D006EC35F002D05C
:1008600000EC35F040EC36F0D1EC37F003E36AEC05
:1008700030F007D031AE05D02D6A2E6A2F6A306A6B
:10088000316A2DC062F22EC063F22FC064F230C014
:1008900065F231C066F2596AAFEC1FF0E80E886F5E
:1008A000030E896F3D803F823E86C2D73DA00BD0AC
:1008B000886709D0896707D03D9055EC21F03F92B9
:1008C0003D9C3AEC23F025EC02F0E2EC0AF01BEC44
:1008D0000BF054EC0BF021EC01F0F1EC00F079ECB2
:1008E00001F0020E9C6328D057EC00F020E3186A58
:1008F000196A1A6A1B6A1C6A18C030F219C031F2F0
:100900001AC032F21BC033F21CC034F2C9EC36F00C
:1009100032C02BF233C02CF234C02DF235C02EF28F
:1009200036C02FF2916B926B976B986B20D07AEC5C
:1009300000F063EC00F01BD07AEC00F057EC00F014
:1009400014E3186A196A1A6A1B6A1C6A18C030F222
:1009500019C031F21AC032F21BC033F21CC034F29B
:10096000916B926B976B986B02D063EC00F03F9A9F
:100970009D6705D095EC03F03D983F8A06D0010EA7
:100980009D6303D0A0EC03F03D988EEC01F09E67D0
:1009900004D04DEC03F03D8A22D0010E9E6304D0BA
:1009A00040EC03F03D8A1BD0020E9E6304D022EC83
:1009B00003F03D8A14D0030E9E6304D07DEC03F057
:1009C0003D9A0DD0040E9E6304D06EEC03F03D9A68
:1009D00006D0050E9E6303D05FEC03F03D9ABCEC9D
:1009E00001F03DA607D082EC25F036EC26F0E7ECCE
:1009F00021F03D966CC018F06DC019F0180618284B
:100A0000D8B41906D8B418521950735D02E11850C1
:100A1000725DD8B02CD06CC072F06DC073F062C043
:100A20006FF063C070F067C074F068C075F02BC2DF
:100A300044F22CC245F22DC246F22EC247F22FC21A
:100A400048F230C249F231C24AF232C24BF233C2EA
:100A50004CF234C24DF200C28AF001C28BF0B6698A
:100A60003E803E82020E9C6101D03E8440D08A6767
:100A70003ED08B673CD0B6670FD00A0E186E000EC2
:100A8000196E1850725F1950735B73AF04D0185011
:100A9000725F1950735B07D0B60772077229D8B41A
:100AA0007307D8B4725362C06FF063C070F067C050
:100AB00074F068C075F02BC244F22CC245F22DC20E
:100AC00046F22EC247F22FC248F230C249F231C27A
:100AD0004AF232C24BF233C24CF234C24DF2B66724
:100AE00006D03E803E82020E9C6101D03E84795148
:100AF0006D5D02E178516C5DD8A00FD06CC078F0CC
:100B00006DC079F062C076F063C077F067C07AF0AC
:100B100068C07BF002C28DF00ED08D6712D06CC021
:100B200078F06DC079F062C076F063C077F067C08E
:100B30007AF068C07BF011EC01F0E1EC00F069ECB8
:100B400001F045EC20F02BE3B9EC1FF0010E4462FC
:100B500007D03DB013D0596AC8EC06F0596A1FD0CF
:100B6000020E44620ED0596A3D7CE80E886F030E77
:100B7000896F3D80596A3E863F8211D0886B896BB0
:100B80000ED00B0E446207D03DB009D0596A0BEC71
:100B900008F0596A04D00C0E446201D0596AA56766
:100BA00002D08AEC02F0010EA56302D071EC02F0D3
:100BB000020EA56302D09AEC02F0030EA56302D0E8
:100BC000BAEC02F0040EA56302D0D6EC02F0050EDA
:100BD000A56302D0E5EC02F020EC23F067C218F028
:100BE00068C219F07351195C02E17251185CD8B0F7
:100BF00011D072C067F273C068F26FC069F270C042
:100C00006AF274C06BF275C06CF2A3C08EF0A4C01F
:100C10008FF012D08F6710D08E670ED0186A196AC5
:100C200018C067F219C068F218C069F219C06AF2F8
:100C300018C06BF219C06CF23DA205D03D923E8007
:100C40003E823E843E86904F9089010E90630CD088
:100C500099519F5DD8B408D09FC099F03BEC22F029
:100C6000020E9C6301D03E84020E906300D0030EFE
:100C7000906305D03EA603D03E9660EC1FF0040EB4
:100C8000906305D03EA403D03E9438EC1EF0050ED0
:100C9000906305D03EA203D03E928EEC1DF0060E6E
:100CA000906305D03EA003D03E9000EC1DF0070EEF
:100CB00090635CD0020E9C6338D05DEC00F030E3B2
:100CC000186A196A1A6A1B6A1C6A18C030F219C0BD
:100CD00031F21AC032F21BC033F21CC034F218C019
:100CE00049F219C04AF21AC04BF21BC04CF21CC0A8
:100CF0004DF2C9EC36F032C02BF233C02CF234C0C6
:100D00002DF235C02EF236C02FF232C044F233C07D
:100D100045F234C046F235C047F236C048F226D01C
:100D20007AEC00F063EC00F021D07AEC00F05DEC9E
:100D300000F01AE3186A196A1A6A1B6A1C6A18C05A
:100D400030F219C031F21AC032F21BC033F21CC0AB
:100D500034F218C049F219C04AF21AC04BF21BC053
:100D60004CF21CC04DF202D063EC00F0080E906310
:100D700002D059EC01F0090E906303D03EB0D1ECE3
:100D800000F00A0E906302D001EC01F018EF04F0BD
:100D9000010EA76F55EC21F09FEC21F0000EF86ECC
:100DA000520EF76E780EF66EB9EC21F09A6B05ECE8
:100DB00007F0F6EC07F00DE006E29A2B060E9A65B6
:100DC00001D09A6B05D09A079AAF02D0060E9A6F9F
:100DD000EED745EC20F012E3B9EC1FF0030E4460AF
:100DE0000ED0010E446203D0D2EC07F008D0020E00
:100DF000446204D0596AD2EC07F001D0DAD79FECF4
:100E000021F03D82A76B446A120055EC21F09A67ED
:100E100018D0000EF86E520EF76E8E0EF66EB9EC0C
:100E200021F0000EF86E520EF76EA40EF66EB9ECBD
:100E300021F0000EF86E520EF76EBA0EF66EB9EC97
:100E400021F0010E9A6318D0000EF86E520EF76E64
:100E5000FC0EF66EB9EC21F0000EF86E530EF76E34
:100E6000120EF66EB9EC21F0000EF86E530EF76E0E
:100E7000280EF66EB9EC21F0020E9A6318D0000E1F
:100E8000F86E530EF76ED80EF66EB9EC21F0000E28
:100E9000F86E530EF76EEE0EF66EB9EC21F0000E02
:100EA000F86E540EF76E040EF66EB9EC21F0030ED8
:100EB0009A6318D0000EF86E540EF76E880EF66E18
:100EC000B9EC21F0000EF86E540EF76E9E0EF66E21
:100ED000B9EC21F0000EF86E540EF76EB40EF66EFB
:100EE000B9EC21F0040E9A6318D0000EF86E550E7E
:100EF000F76EA60EF66EB9EC21F0000EF86E530EEA
:100F0000F76EEE0EF66EB9EC21F0000EF86E540E90
:100F1000F76E040EF66EB9EC21F0050E9A6318D048
:100F2000000EF86E550EF76ED20EF66EB9EC21F08B
:100F3000000EF86E540EF76E9E0EF66EB9EC21F0B0
:100F4000000EF86E540EF76EB40EF66EB9EC21F08A
:100F5000060E9A6326D0010EA06308D0000EF86E2C
:100F6000560EF76E400EF66EB9EC21F0020EA0633D
:100F700008D0000EF86E560EF76E820EF66EB9ECC3
:100F800021F0000EF86E560EF76E560EF66EB9ECA6
:100F900021F0000EF86E560EF76E6C0EF66EB9EC80
:100FA00021F012009A6702D06CEF18F0010E9A63DC
:100FB00002D09DEF19F0020E9A6302D01BEF1AF0D7
:100FC000030E9A6302D088EF1AF0040E9A6302D0DF
:100FD00044EF1BF0050E9A6302D0B0EF1BF0060E33
:100FE0009A6302D071EF1CF09FEF21F0595211E08B
:100FF00059AE08D05950E86CFE0B0BE0596AD894F2
:10100000D88008D05950FE0B04E0596AD894D89083
:1010100001D0D88412003E8C010EA76F9FEC21F006
:10102000000EF86E560EF76EC40EF66EB9EC21F097
:1010300049EC08F0F6EC07F00DE006E29B2B140EED
:101040009B6501D09B6B05D09B079BAF02D0140E14
:101050009B6FEED745EC20F013E3B9EC1FF0030EC5
:1010600044600FD0010E446204D0596A76EC0AF055
:1010700008D0020E446204D0596A76EC0AF001D01E
:10108000D9D79FEC21F0596A3D82A76B446A3E9CF8
:10109000120055EC21F09B670CD0000EF86E560E36
:1010A000F76EDA0EF66EB9EC21F0D9EC27F0D7EC3A
:1010B00027F0010E9B6318D0000EF86E560EF76EE7
:1010C000F00EF66EB9EC21F0000EF86E570EF76ECA
:1010D000060EF66EB9EC21F0000EF86E570EF76EA4
:1010E0001C0EF66EB9EC21F0020E9B6318D0000EB8
:1010F000F86E570EF76E320EF66EB9EC21F0000E58
:10110000F86E570EF76E060EF66EB9EC21F0000E73
:10111000F86E570EF76E480EF66EB9EC21F0030E1E
:101120009B6318D0000EF86E570EF76E5E0EF66ECB
:10113000B9EC21F0000EF86E570EF76E740EF66ED5
:10114000B9EC21F0000EF86E570EF76E8A0EF66EAF
:10115000B9EC21F0040E9B6318D0000EF86E570E08
:10116000F76EEC0EF66EB9EC21F0000EF86E580E2C
:10117000F76E020EF66EB9EC21F0000EF86E580E06
:10118000F76E180EF66EB9EC21F0050E9B6318D0C1
:10119000000EF86E580EF76E440EF66EB9EC21F0A4
:1011A000000EF86E580EF76E5A0EF66EB9EC21F07E
:1011B000000EF86E580EF76E700EF66EB9EC21F058
:1011C000060E9B6318D0000EF86E580EF76E9C0E3C
:1011D000F66EB9EC21F0000EF86E580EF76EB20EF6
:1011E000F66EB9EC21F0000EF86E580EF76EC80ED0
:1011F000F66EB9EC21F0070E9B6318D0000EF86E66
:10120000580EF76EDE0EF66EB9EC21F0000EF86E99
:10121000580EF76EB20EF66EB9EC21F0000EF86EB5
:10122000580EF76EC80EF66EB9EC21F0080E9B63EF
:1012300018D0000EF86E580EF76EF40EF66EB9EC7C
:1012400021F0000EF86E590EF76E0A0EF66EB9EC2C
:1012500021F0000EF86E590EF76E200EF66EB9EC06
:1012600021F0090E9B6318D0000EF86E590EF76E30
:10127000A40EF66EB9EC21F0000EF86E590EF76E62
:10128000BA0EF66EB9EC21F0000EF86E590EF76E3C
:10129000D00EF66EB9EC21F00A0E9B6318D0000E4A
:1012A000F86E5A0EF76E1C0EF66EB9EC21F0000EB9
:1012B000F86E5A0EF76E320EF66EB9EC21F0000E93
:1012C000F86E5A0EF76E480EF66EB9EC21F00B0E62
:1012D0009B6318D0000EF86E5A0EF76E980EF66EDD
:1012E000B9EC21F0000EF86E5A0EF76EAE0EF66EE7
:1012F000B9EC21F0000EF86E5A0EF76EC40EF66EC1
:10130000B9EC21F00C0E9B6318D0000EF86E5B0E4A
:10131000F76E140EF66EB9EC21F0000EF86E5B0E4F
:10132000F76E2A0EF66EB9EC21F0000EF86E5B0E29
:10133000F76E400EF66EB9EC21F00D0E9B6318D0DF
:10134000000EF86E5B0EF76E8A0EF66EB9EC21F0A9
:10135000000EF86E5B0EF76EA00EF66EB9EC21F083
:10136000000EF86E5B0EF76EB60EF66EB9EC21F05D
:101370000E0E9B6318D0000EF86E5B0EF76ECC0E4F
:10138000F66EB9EC21F0000EF86E5B0EF76EA00E53
:10139000F66EB9EC21F0000EF86E5B0EF76EB60E2D
:1013A000F66EB9EC21F00F0E9B6318D0000EF86EAC
:1013B0005B0EF76EE20EF66EB9EC21F0000EF86EE1
:1013C0005B0EF76EF80EF66EB9EC21F0000EF86EBB
:1013D0005C0EF76E0E0EF66EB9EC21F0100E9B63EC
:1013E00018D0000EF86E5C0EF76E580EF66EB9EC63
:1013F00021F0000EF86E5C0EF76E6E0EF66EB9EC14
:1014000021F0000EF86E5C0EF76E840EF66EB9ECED
:1014100021F0110E9B6318D0000EF86E5C0EF76E73
:10142000B00EF66EB9EC21F0000EF86E5C0EF76EA1
:101430006E0EF66EB9EC21F0000EF86E5C0EF76ED3
:10144000840EF66EB9EC21F0120E9B6318D0000EDC
:10145000F86E5C0EF76EDC0EF66EB9EC21F0000E45
:10146000F86E5D0EF76E080EF66EB9EC21F0000E08
:10147000F86E5D0EF76E1E0EF66EB9EC21F0130ECF
:101480009B6318D0000EF86E5D0EF76E460EF66E7A
:10149000B9EC21F0000EF86E5D0EF76E720EF66E6E
:1014A000B9EC21F0000EF86E5D0EF76E880EF66E48
:1014B000B9EC21F0140E9B6318D0000EF86E5D0E8F
:1014C000F76EAA0EF66EB9EC21F0000EF86E5D0E06
:1014D000F76EC00EF66EB9EC21F0000EF86E5D0EE0
:1014E000F76ED60EF66EB9EC21F012009FEC21F0EB
:1014F0009B6701D064D0010E9B6302D0BFEF0CF05C
:10150000020E9B6302D0AAEF0DF0030E9B6302D084
:10151000FAEF0FF0040E9B6302D05BEF11F0050EA3
:101520009B6302D0E8EF11F0060E9B6302D066EFDA
:1015300012F0070E9B6302D0E4EF12F0080E9B63DB
:1015400002D067EF13F0090E9B6302D0D0EF13F0C7
:101550000A0E9B6302D03DEF14F00B0E9B6302D08A
:10156000FBEF14F00C0E9B6302D073EF15F00D0E21
:101570009B6302D02EEF0CF00E0E9B6302D04EEF59
:101580000CF00F0E9B6302D023EF16F0100E9B633E
:1015900002D0C9EF16F0110E9B6302D023EF17F0B3
:1015A000120E9B6302D07DEF17F0130E9B6302D0E7
:1015B000C6EF17F0140E9B6302D0FBEF17F03D82CD
:1015C0009FEF21F03FA631D0D89062376337643760
:1015D000D890623763376437D8906237633764379F
:1015E00033EC30F060C018F061C019F01850622779
:1015F000195063231A50642341EC30F062C018F094
:1016000063C019F064C01AF0090E1D6EA9EC38F021
:1016100018C062F019C063F01AC064F0040E1D64B3
:1016200003D0622BD8B4632B05D0646B60C062F02A
:1016300061C063F012003FA431D0D8906C376D3791
:101640006E37D8906C376D376E37D8906C376D37F2
:101650006E3733EC30F06AC018F06BC019F01850D8
:101660006C2719506D231A506E2341EC30F06CC07A
:1016700018F06DC019F06EC01AF0090E1D6EA9ECBD
:1016800038F018C06CF019C06DF01AC06EF0040E7E
:101690001D6403D06C2BD8B46D2B05D06E6B6AC063
:1016A0006CF06BC06DF012003FA831D0D890673756
:1016B00068376937D890673768376937D8906737A0
:1016C0006837693733EC30F065C018F066C019F040
:1016D00018506727195068231A50692341EC30F0DD
:1016E00067C018F068C019F069C01AF0090E1D6EC5
:1016F000A9EC38F018C067F019C068F01AC069F09A
:10170000040E1D6403D0672BD8B4682B05D0696B19
:1017100065C067F066C068F01200530EA7EC21F0B8
:10172000200E3DAE3C0EDBEC20F0270EA7EC21F0A6
:10173000200E3DBE3C0EDBEF20F0000EF86E500E8A
:10174000F76EB40EF66EB9EC21F041EC30F006C243
:1017500018F007C219F095EC3AF074EC39F052EC3D
:1017600021F0A86702D0490E09D0010EA86302D06B
:10177000480E04D0020EA86301D0470EA7EF21F057
:10178000A86B010EA76F3DBE09D0000EF86E500E7B
:10179000F76E700EF66EB9EC21F008D0000EF86E00
:1017A000500EF76E860EF66EB9EC21F0000EF86E54
:1017B000520EF76E620EF66EB9EC21F0000EF86E66
:1017C000500EF76EBC0EF66EB9EC21F09DEC0BF0EE
:1017D00059522BE006C218F007C219F0A86705D0CD
:1017E000010E1D6E000E1E6E0FD0010EA86305D0F7
:1017F0000A0E1D6E000E1E6E07D0020EA86304D0E6
:10180000640E1D6E000E1E6E59BE05D01D501826AA
:101810001E50192204D01D50185E1E50195A18C0AF
:1018200006F219C007F2596AAED745EC20F0D0E3B2
:10183000B9EC1FF0020E446206D0A82B030EA86379
:1018400001D0A86BA0D70B0E446202D0D88005D07F
:10185000010E446202D0D89000D012006DEC0CF062
:101860009FEC21F03D9E040E186E100E196E18C0EC
:1018700006F219C007F284DF10E23D8E06C204F2C0
:1018800007C205F2FC0E186E080E196E18C006F29B
:1018900019C007F275DF01E2C4D012006DEC0CF044
:1018A0009FEC21F03D9E040E186E100E196E18C0AC
:1018B00006F219C007F264DFF0E23D8E06C204F2C0
:1018C00007C205F2FC0E186E080E196E18C006F25B
:1018D00019C007F255DFE1E28CD108C26DF209C2EE
:1018E0006EF20AC26FF20BC270F20CC271F20DC23C
:1018F00072F20EC273F20FC274F210C275F211C20C
:1019000076F212C277F213C278F214C279F215C2DB
:101910007AF216C27BF217C27CF218C27DF219C2AB
:101920007EF21AC27FF21BC280F212006DC208F270
:101930006EC209F26FC20AF270C20BF271C20CF2EF
:1019400072C20DF273C20EF274C20FF275C210F2BF
:1019500076C211F277C212F278C213F279C214F28F
:101960007AC215F27BC216F27CC217F27DC218F25F
:101970007EC219F27FC21AF280C21BF212003F86A9
:101980003F846DEC0CF03E8855EC21F09FEC21F08B
:10199000000EF86E510EF76ED20EF66EB9EC21F015
:1019A000000EF86E520EF76E360EF66EB9EC21F0A0
:1019B000626B636B646BAAD945EC20F0FCE3B9EC75
:1019C0001FF0010E446284D062C004F263C005F2CD
:1019D0009FEC21F0000EF86E510EF76EE80EF66ED9
:1019E000B9EC21F0000EF86E520EF76E360EF66E60
:1019F000B9EC21F0626B636B646B88D945EC20F025
:101A0000FCE3B9EC1FF0010E446262D062C006F242
:101A100063C007F27ED850EC20F050EC20F03F96E7
:101A20003F949FEC21F0000EF86E510EF76EFE0E03
:101A3000F66EB9EC21F044D92DC008F22EC009F29F
:101A40002FC00AF230C00BF231C00CF259D92DC0B0
:101A50000DF22EC00EF22FC00FF230C010F231C0C6
:101A600011F29AD950EC20F0000EF86E520EF76E7B
:101A7000620EF66EB9EC21F0B9EC1FF0010E446273
:101A800027D09FEC21F0B2D950EC20F0000EF86E78
:101A9000520EF76E620EF66EB9EC21F0B9EC1FF043
:101AA000010E446215D09FEC21F058DA50EC20F082
:101AB000000EF86E520EF76E620EF66EB9EC21F063
:101AC000B9EC1FF0010E446203D05DEC23F004D0AA
:101AD00096EC0CF06DEC0DF01200000EF86E5E0E40
:101AE000F76E5C0EF66EB9EC21F0000EF86E5E0E2D
:101AF000F76E720EF66EB9EC21F0000EF86E5E0E07
:101B0000F76E880EF66EB9EC21F050EC20F09FEFE6
:101B100021F0000EF86E5E0EF76EB40EF66EB9ECA4
:101B200021F0000EF86E5E0EF76ECA0EF66EB9EC7E
:101B300021F0000EF86E5E0EF76EE00EF66EB9EC58
:101B400021F0000EF86E5E0EF76EF60EF66EB9EC32
:101B500021F012003F886DEC0CF055EC21F09FEC69
:101B600021F0000EF86E510EF76ED20EF66EB9EC43
:101B700021F0000EF86E520EF76E360EF66EB9ECCE
:101B800021F0676B686B696BE4D845EC20F0FCE3EF
:101B9000B9EC1FF0010E446283D067C004F268C044
:101BA00005F29FEC21F0000EF86E510EF76EE80E74
:101BB000F66EB9EC21F0000EF86E520EF76E360E8E
:101BC000F66EB9EC21F0676B686B696BC2D845ECB7
:101BD00020F0FCE3B9EC1FF0010E446261D067C055
:101BE00006F268C007F295DF50EC20F050EC20F0D0
:101BF0003F989FEC21F0000EF86E520EF76E140E17
:101C0000F66EB9EC21F05CD82DC012F22EC013F2A2
:101C10002FC014F230C015F231C016F271D82DC0A9
:101C200017F22EC018F22FC019F230C01AF231C0CC
:101C30001BF2B2D850EC20F0000EF86E520EF76E88
:101C4000620EF66EB9EC21F0B9EC1FF0010E4462A1
:101C500027D09FEC21F000D950EC20F0000EF86E58
:101C6000520EF76E620EF66EB9EC21F0B9EC1FF071
:101C7000010E446215D09FEC21F024D950EC20F0E5
:101C8000000EF86E520EF76E620EF66EB9EC21F091
:101C9000B9EC1FF0010E446203D064EC23F004D0D1
:101CA00096EC0CF06DEC0DF01200000EA7EC21F09C
:101CB000F6EC3AF01EEC3BF050EC20F0B9EF1FF0E0
:101CC00004C218F005C219F0A7EC32F02DEC34F084
:101CD00004EC31F006C218F007C219F0A7EC32F09C
:101CE00038EC34F000EC35F080EC30F01E0E186E5D
:101CF000AEEC32F02DEC34F054EC30F0C3EF34F0B5
:101D000096EC30F043EC34F0317E120055EC21F0CB
:101D10005CEC20F005EC02F0E2EC0AF0000EF86E4C
:101D2000510EF76EAE0EF66EB9EC21F062C018F0EF
:101D300063C019F064C01AF0A1EC32F02DEC34F05D
:101D4000ADEC3AF0050E376E386A4FEC3AF0A0EF82
:101D500039F055EC21F05CEC20F0E5EC01F054ECAE
:101D60000BF0000EF86E510EF76EC60EF66EB9EC63
:101D700021F067C018F068C019F069C01AF0A1EC32
:101D800032F02DEC34F0ADEC3AF0050E376E386AD7
:101D90004FEC3AF0A0EF39F055EC21F0000EF86E60
:101DA000500EF76E9C0EF66EB9EC21F041EC30F05F
:101DB00004C218F005C219F095EC3AF0040E376E23
:101DC00074EC39F0000EF86E500EF76EA80EF66E39
:101DD000B9EC21F041EC30F006C218F007C219F05E
:101DE00095EC3AF0040E376E74EF39F055EC21F0B3
:101DF000000EF86E510EF76EFE0EF66EB9EC21F085
:101E0000000EF86E520EF76E2A0EF66EB9EC21F047
:101E100008C22DF009C22EF00AC22FF00BC230F01A
:101E20000CC231F0F6EC3AF01EEC3BF0000EF86E0E
:101E3000520EF76E300EF66EB9EC21F00DC22DF099
:101E40000EC22EF00FC22FF010C230F011C231F0CE
:101E5000F6EC3AF01EEF3BF055EC21F0000EF86E78
:101E6000520EF76E140EF66EB9EC21F0000EF86EFD
:101E7000520EF76E2A0EF66EB9EC21F012C22DF05A
:101E800013C22EF014C22FF015C230F016C231F07A
:101E9000F6EC3AF01EEC3BF0000EF86E520EF76EC8
:101EA000300EF66EB9EC21F017C22DF018C22EF0EC
:101EB00019C22FF01AC230F01BC231F0F6EC3AF022
:101EC0001EEF3BF055EC21F0000EF86E520EF76E4F
:101ED000140EF66EB9EC21F0000EF86E520EF76E8D
:101EE0002A0EF66EB9EC21F012C218F013C219F0E6
:101EF00014C21AF015C21BF016C21CF01C50B0EC34
:101F000021F01B50B0EC21F01A50B0EC21F0195028
:101F1000B0EC21F01850B0EC21F0000EF86E520E2B
:101F2000F76E300EF66EB9EC21F017C218F018C239
:101F300019F019C21AF01AC21BF01BC21CF01C5077
:101F4000B0EC21F01B50B0EC21F01A50B0EC21F0B5
:101F50001950B0EC21F01850B0EF21F055EC21F001
:101F6000000EF86E510EF76EFE0EF66EB9EC21F013
:101F7000000EF86E520EF76E2A0EF66EB9EC21F0D6
:101F800008C218F009C219F00AC21AF00BC21BF0FD
:101F90000CC21CF01C50B0EC21F01B50B0EC21F036
:101FA0001A50B0EC21F01950B0EC21F01850B0EC00
:101FB00021F0000EF86E520EF76E300EF66EB9EC90
:101FC00021F00DC218F00EC219F00FC21AF010C2A3
:101FD0001BF011C21CF01C50B0EC21F01B50B0ECF7
:101FE00021F01A50B0EC21F01950B0EC21F018504B
:101FF000B0EF21F055EC21F0A86B9FEC21F0A2A9E5
:1020000009D0000EF86E570EF76EB60EF66EB9ECEC
:1020100021F008D0000EF86E570EF76EA00EF66E87
:10202000B9EC21F0000EF86E570EF76ECC0EF66E7E
:10203000B9EC21F0000EF86E520EF76E360EF66E09
:10204000B9EC21F05DC22DF05EC22EF05FC22FF020
:1020500060C230F061C231F05DC24AF05EC24BF046
:102060005FC24CF060C24DF061C24EF0E4EC3BF058
:10207000C3EC34F000EC36F000EC37F0C4EC31F097
:1020800012EC37F02DC045F02EC046F02FC047F0BF
:1020900030C048F031C049F0596A52EC21F0000ECE
:1020A000F86E570EF76EE20EF66EB9EC21F045C0F1
:1020B0002DF046C02EF047C02FF048C030F049C088
:1020C00031F0ADEC3AF0030E376E010E386E4FEC86
:1020D0003AF0A0EC39F0000EF86E570EF76EE80EED
:1020E000F66EB9EC21F045C02DF046C02EF047C089
:1020F0002FF048C030F049C031F083EC37F0E4EC09
:102100003BF043EC34F0ADEC3AF0050E376E030EC5
:10211000386E4FEC3AF0A0EC39F0000EF86E600E1D
:10212000F76E5E0EF66EBCEC21F0A86702D01B0EB7
:1021300004D0010EA86301D0190EA7EC21F0A86706
:1021400002D0BEEC36F0010EA86302D05EEC36F091
:10215000F6EC07F02DE00DE245C02DF046C02EF064
:1021600047C02FF048C030F049C031F006EC35F0E0
:1021700013D045C02DF046C02EF047C02FF048C008
:1021800030F049C031F000EC35F05EEC36F0A1ECF7
:1021900037F002E36AEC30F02DC045F02EC046F077
:1021A0002FC047F030C048F031C049F0596A77D7A6
:1021B00045EC20F0C4E3B9EC1FF0010E44621DD0E1
:1021C00045C02DF046C02EF047C02FF048C030F07B
:1021D00049C031F083EC37F0E4EC3BF043EC34F0F1
:1021E0002DC05DF22EC05EF22FC05FF230C060F2F3
:1021F00031C061F256EC23F016D0020E446206D0D4
:10220000A82B020EA8634BD7A86B49D7020E4464D3
:1022100046D74AC05DF24BC05EF24CC05FF24DC083
:1022200060F26DEC0DF012002DEC34F015EC37F08F
:10223000420E366E700E356E326A336A346AC3EC03
:1022400034F0ADEC3AF0030E376E010E386E4FEC01
:102250003AF0A0EC39F0000EF86E5F0EF76E9A0EB1
:10226000F66EBCEC21F012002DEC34F015EC37F0DA
:10227000ADEC3AF0040E376E020E386E0AD02DEC3B
:1022800034F015EC37F0ADEC3AF0040E376E010E79
:10229000386E4FEC3AF0A0EC39F0000EF86E5F0E9D
:1022A000F76E960EF66EBCEC21F01200200EA7EC35
:1022B00021F052EF21F000C245F001C246F055EC8A
:1022C00021F0000EF86E580EF76E2E0EF66EB9EC79
:1022D00021F0000EF86E5F0EF76E2E0EF66EB9EC62
:1022E00021F0000EF86E520EF76E360EF66EB9EC57
:1022F00021F0000EF86E5F0EF76E440EF66EB9EC2C
:1023000021F000C218F001C219F0A7EC32F0B7DFDB
:10231000CDDFF6EC07F03EE01CE200C218F001C28F
:1023200019F00A0E1D6E000E1E6E1D5018261E504E
:102330001922E80E1D6E030E1E6E19501E5C02E17E
:1023400018501D5CD8B004D01DC018F01EC019F084
:102350001BD000C218F001C219F00A0E1D6E000E4B
:102360001E6E1D50185E1E50195A320E1D6E000E44
:102370001E6E19501E5C02E118501D5CD8A004D0DE
:102380001DC018F01EC019F018C000F219C001F2EB
:10239000596A95D745EC20F0BCE3B9EC1FF055EC39
:1023A00021F0030E446006D0010E446203D0D1EC4C
:1023B00024F006D045C000F246C001F26DEC0DF0ED
:1023C00012004D0E3DBE230EA7EC21F052EF21F07E
:1023D000020EA76F3D9E03C245F055EC21F0000EA2
:1023E000F86E580EF76E860EF66EB9EC21F0000E00
:1023F000F86E520EF76E4C0EF66EB9EC21F0000E30
:10240000F86E5F0EF76E720EF66EB9EC21F003C235
:1024100018F0AEEC32F028DF000EF86E5F0EF76EAB
:102420007E0EF66EB9EC21F0780EA2A7200EDBEC42
:1024300020F0000EF86E510EF76E440EF66EBCECF6
:1024400021F08DEC0BF0BDDF3DBE17D0F6EC07F0B0
:102450001AE009E203C218F0182AFA0E186402D032
:10246000FA0E186E07D003C218F01806186602D0CC
:10247000010E186E18C003F204D0F6EC07F003E06A
:10248000A277596AAAD745EC20F0DEE355EC21F09B
:10249000B9EC1FF0010E446205D0E3EC24F0F5EC3A
:1024A00024F013D0020E446202D03D7E96D70B0E6C
:1024B000446202D03D7E91D70C0E446206D045C0E6
:1024C00003F246C004F26DEC0DF0120055EC21F061
:1024D0000DC22DF00EC22EF00FC22FF010C230F040
:1024E00011C231F008C232F009C233F00AC234F02E
:1024F0000BC235F00CC236F0C3EC34F0317ED3ECB5
:1025000031F00EC004F20FC005F20DC22DF00EC264
:102510002EF00FC22FF010C230F011C231F01E0E9B
:10252000186EAEEC32F038EC34F006EC35F008C240
:1025300032F009C233F00AC234F00BC235F00CC2DB
:1025400036F0C3EC34F0317ED3EC31F00EC006F23D
:102550000FC007F29FEC21F0000EF86E510EF76EDF
:10256000FE0EF66EB9EC21F0CCEC0EF050EC20F043
:10257000000EF86E520EF76E620EF66EB9EC21F098
:10258000B9EC1FF09FEC21F0F6EC0EF050EC20F0CF
:10259000000EF86E520EF76E620EF66EB9EC21F078
:1025A000B9EC1FF09FEC21F0AEEC0FF050EC20F0F6
:1025B000000EF86E520EF76E620EF66EB9EC21F058
:1025C000B9EC1FF09FEF21F055EC21F017C22DF070
:1025D00018C22EF019C22FF01AC230F01BC231F00F
:1025E00012C232F013C233F014C234F015C235F007
:1025F00016C236F0C3EC34F0317ED3EC31F00EC0AD
:1026000004F20FC005F217C22DF018C22EF019C245
:102610002FF01AC230F01BC231F01E0E186EAEEC55
:1026200032F038EC34F006EC35F012C232F013C25E
:1026300033F014C234F015C235F016C236F0C3ECD4
:1026400034F0317ED3EC31F00EC006F20FC007F249
:102650009FEC21F0000EF86E520EF76E140EF66E1F
:10266000B9EC21F0CCEC0EF050EC20F0000EF86E3E
:10267000520EF76E620EF66EB9EC21F0B9EC1FF057
:102680009FEC21F02CEC0FF050EC20F0000EF86ED7
:10269000520EF76E620EF66EB9EC21F0B9EC1FF037
:1026A0009FEC21F062EC0FF050EC20F0000EF86E81
:1026B000520EF76E620EF66EB9EC21F0B9EC1FF017
:1026C0009FEF21F0150EA7EC21F052EF21F0A0C0F2
:1026D00045F055EC21F09FEC21F0000EF86E590EFC
:1026E000F76E360EF66EB9EC21F0000EF86E590E4C
:1026F000F76E4C0EF66EB9EC21F0000EF86E520E2D
:10270000F76E360EF66EB9EC21F0A06708D0000E19
:10271000F86E590EF76E620EF66EB9EC21F0010EEE
:10272000A06308D0000EF86E590EF76E780EF66EA4
:10273000B9EC21F0020EA06308D0000EF86E590E1D
:10274000F76E8E0EF66EB9EC21F0BCDFF6EC07F0FA
:102750000DE006E2A02B020EA06501D0A06B05D013
:10276000A007A0AF02D0020EA06FCFD745EC20F09B
:10277000ECE355EC21F0B9EC1FF0030E446006D0F9
:10278000010E446203D0D3EC23F004D045C0A0F086
:102790006DEC0DF012001B0EA7EC21F052EF21F0B2
:1027A000A1C045F055EC21F09FEC21F0A06713D0BB
:1027B000000EF86E5E0EF76E5C0EF66EB9EC21F050
:1027C000000EF86E5E0EF76E9E0EF66EB9EC21F0FE
:1027D00050EC20F051D0000EF86E590EF76EE60E58
:1027E000F66EB9EC21F0000EF86E590EF76EFC0E85
:1027F000F66EB9EC21F0000EF86E520EF76E360E42
:10280000F66EB9EC21F055EC21F0000EF86E5A0E80
:10281000F76E120EF66EB9EC21F041EC30F0A1C06B
:1028200018F095EC3AF0010E376E74EC39F0B3DF26
:10283000F6EC07F00DE006E2A12B070EA16501D032
:10284000A16B05D0A107A1AF02D0070EA16FDBD706
:1028500045EC20F0EDE355EC21F0B9EC1FF0030E50
:10286000446006D0010E446203D0C1EC23F004D0D2
:1028700045C0A1F06DEC0DF0120055EC21F09FEC7D
:1028800021F0000EF86E5A0EF76E5E0EF66EB9EC81
:1028900021F0000EF86E5A0EF76E740EF66EB9EC5B
:1028A00021F0000EF86E520EF76E620EF66EB9EC65
:1028B00021F07C6B7F6B3D983D9A82EC25F036ECE5
:1028C00026F0E7EC21F0916B926B1FEC23F0976BF5
:1028D000986B20EC23F0000EF86E5A0EF76E8A0EFD
:1028E000F66EB9EC21F041EC30F07CC018F095ECBC
:1028F0003AF0020E376E74EC39F0000EF86E5A0E94
:10290000F76E920EF66EB9EC21F041EC30F097C004
:1029100018F098C019F095EC3AF0040E376E74EC8C
:1029200039F0F6EC07F03AE00AE27C2B7F2B140E2C
:102930007C6504D0140E7C6F140E7F6F06D07C076C
:102940007F077CAF02D07C6B7F6B3D983D9A82EC19
:1029500025F036EC26F0E7EC21F07CC018F0AEEC68
:1029600032F02DEC34F0420E366E4C0E356E990E70
:10297000346E990E336E9A0E326E43EC34F0D3EC13
:1029800031F00EC091F00FC092F01FEC23F00EC09A
:1029900097F00FC098F020EC23F09DD745EC20F085
:1029A000C0E3B9EC1FF0030E446008D0010E44628E
:1029B00001D005D0020E446201D001D08CD79FEC2B
:1029C00021F07C6B7F6B3D983D9A82EC25F036ECD4
:1029D00026F0E7EC21F0916B926B1FEC23F0976BE4
:1029E000986B3D8220EF23F04F0E3DBE230EA7ECE7
:1029F00021F052EF21F055EC21F09FEC21F03D9EAB
:102A0000A2C045F055EC21F0020EA76F000EF86E43
:102A10005A0EF76EDA0EF66EB9EC21F0000EF86E73
:102A2000520EF76E4C0EF66EB9EC21F0000EF86EF9
:102A30005A0EF76EF00EF66EB9EC21F0780EA2A1E8
:102A4000200EDBEC20F0000EF86E510EF76E440EF7
:102A5000F66EBCEC21F0000EF86E5B0EF76E020E07
:102A6000F66EB9EC21F0780EA2A3200EDBEC20F07C
:102A7000000EF86E510EF76E440EF66EBCEC21F0AF
:102A80008DEC0BF0B1DFF6EC07F005E03DAEA27186
:102A90003DBEA273B7D745EC20F0F5E355EC21F02D
:102AA000B9EC1FF0010E446203D0F5EC24F011D014
:102AB000020E446202D03D7EA5D70B0E446202D0C6
:102AC0003D7EA0D70C0E446200D045C0A2F06DEC54
:102AD0000DF03D829FEF21F04D0E3DBE230EA7EC81
:102AE00021F052EF21F055EC21F09FEC21F0A2C033
:102AF00045F03D9E020EA76F55EC21F0000EF86EDA
:102B00005B0EF76E560EF66EB9EC21F0000EF86E05
:102B1000520EF76E4C0EF66EB9EC21F0000EF86E08
:102B20005B0EF76E6C0EF66EB9EC21F0A3C018F0D8
:102B3000A4C019F0A7EC32F014EC11F0000EF86EFE
:102B40005B0EF76E780EF66EB9EC21F0780EA2A54A
:102B5000200EDBEC20F0000EF86E510EF76E440EE6
:102B6000F66EBCEC21F08DEC0BF0B6DFA3C018F0D4
:102B7000A4C019F0B80E1D6E0B0E1E6EF6EC07F019
:102B800035E016E23DBE2FD01D5018261E501922EA
:102B9000600E1D6EEA0E1E6E19501E5C02E118508A
:102BA0001D5CD8B004D01DC018F01EC019F015D09F
:102BB0003DBE13D01D50185E1E50195A700E1D6E6A
:102BC000170E1E6E1E50195C02E11D50185CD8B025
:102BD00004D01DC018F01EC019F018C0A3F019C011
:102BE000A4F0596A87D7A275596A84D745EC20F0BA
:102BF000BDE355EC21F0B9EC1FF0010E446209D0A1
:102C0000F5EC24F079EC23F0A3C08EF0A4C08FF093
:102C100011D0020E446202D03D7E6CD70B0E44628E
:102C200002D03D7E67D70C0E446200D045C0A2F0B2
:102C30006DEC0DF012004B0E02D0260E00D0A7EC6A
:102C400021F052EF21F055EC21F09FEC21F002C26F
:102C500045F0A2C046F03D9E020EA76F55EC21F054
:102C6000000EF86E5C0EF76E240EF66EB9EC21F0D5
:102C7000000EF86E520EF76E4C0EF66EB9EC21F0A7
:102C8000000EF86E5C0EF76E3A0EF66EB9EC21F09F
:102C900002C218F0AEEC32F034EC11F0000EF86E17
:102CA0005C0EF76E440EF66EB9EC21F0780EA2AB16
:102CB000200EDBEC20F0000EF86E510EF76E440E85
:102CC000F66EBCEC21F03DAEB6DF3DBEB6DFF6ECF5
:102CD00007F01DE00EE23DAE03D0A27B596ABCD7DF
:102CE00002C218F0182AFA0E186402D0FA0E186EF2
:102CF0000AD03DAE03D0A27B596AAED702C218F00B
:102D0000180618BE186A18C002F2596AA5D745EC11
:102D100020F0DDE355EC21F0B9EC1FF0010E446228
:102D200005D0F5EC24F0BFEC24F013D0020E446281
:102D300002D03D7E91D70B0E446202D03D7E8CD7EF
:102D40000C0E446200D045C002F246C0A2F06DEC09
:102D50000DF01200000EF86E5F0EF76E4E0EF66E5E
:102D6000B9EC21F0AEEC32F02DEC34F06DEC36F035
:102D7000C3EC34F0ADEC3AF0030E376E010E386E52
:102D80004FEC3AF0A0EF39F0230EA7EC21F052EF10
:102D900021F09FEC21F081C245F055EC21F0000EAE
:102DA000F86E5C0EF76E9A0EF66EB9EC21F0000E1E
:102DB000F86E5F0EF76E5C0EF66EB9EC21F0000E49
:102DC000F86E520EF76E360EF66EB9EC21F081C237
:102DD00018F0AAEC16F0D8DFF6EC07F016E081C286
:102DE00018F003E2050E182602D0050E185E0F0E2D
:102DF000186002D00F0E186E640E186402D0640EB4
:102E0000186E18C081F2596AC8D745EC20F0E4E387
:102E100055EC21F0B9EC1FF0030E446006D0010E12
:102E2000446203D007EC25F00CD045C083F246C0C5
:102E300084F247C085F248C086F249C087F26DEC43
:102E40000DF025EF00F09FEC21F082C245F055EC2B
:102E500021F0000EF86E5C0EF76EC60EF66EB9EC41
:102E600021F0000EF86E5F0EF76E5C0EF66EB9EC98
:102E700021F0000EF86E520EF76E360EF66EB9ECBB
:102E800021F082C218F0AAEC16F07EDFF6EC07F013
:102E900016E082C218F003E2050E182602D0050ED5
:102EA000185E0F0E186002D00F0E186E640E1864B4
:102EB00002D0640E186E18C082F2596AC8D745EC69
:102EC00020F0E4E355EC21F0B9EC1FF0030E446070
:102ED00006D0010E446203D019EC25F00CD045C099
:102EE00088F246C089F247C08AF248C08BF249C0D6
:102EF0008CF26DEC0DF033EF00F09FEC21F0A2C0EE
:102F000045F055EC21F0000EF86E5C0EF76EF20EF7
:102F1000F66EB9EC21F0000EF86E5D0EF76E340E11
:102F2000F66EB9EC21F0200EA2BD580EDBEC20F0BD
:102F30005D0EDBEC20F0000EF86E520EF76E360ED2
:102F4000F66EB9EC21F0F6EC07F005E004E2A27DA4
:102F50003BEC22F0D6D745EC20F0F5E3B9EC1FF0BE
:102F6000030E446006D0010E446203D0F5EC24F059
:102F70000CD045C0A2F046C0A3F047C0A4F048C0A2
:102F8000A5F049C0A6F06DEC0DF012009FEC21F009
:102F900055EC21F0000EF86E5D0EF76E5C0EF66ECD
:102FA000B9EC21F0000EF86E520EF76E620EF66E5E
:102FB000B9EC21F0000EF86E5D0EF76E9E0EF66E07
:102FC000B9EC21F041EC30F0B4C018F095EC3AF0D7
:102FD00074EC39F0B9EF1FF0456602D00D0EB56FF5
:102FE000010E456202D00E0EB56F020E456202D090
:102FF0000F0EB56F1200B5C045F09FEC21F055ECF7
:1030000021F0000EF86E5D0EF76EEC0EF66EB9EC68
:1030100021F0000EF86E520EF76E360EF66EB9EC19
:1030200021F0456AD9DF55EC21F0000EF86E5E0EF6
:10303000F76E020EF66EB9EC21F052EC21F0F6ECD0
:1030400007F00EE059AE06D0452A030E456207D0C0
:10305000456A00D0450645AE02D0020E456EE2D765
:1030600045EC20F0ECE355EC21F0B9EC1FF0030E39
:10307000446006D0010E446203D0AFEC23F00CD0C4
:1030800045C0B5F046C0B6F047C0B7F048C0B8F08C
:1030900049C0B9F06DEC0DF012009FEC21F0000E6C
:1030A000F86E5E0EF76E1A0EF66EB9EC21F0000E99
:1030B000F86E5E0EF76E300EF66EB9EC21F0000E73
:1030C000F86E5E0EF76E460EF66EB9EC21F052EC1D
:1030D00020F03D829FEF21F055EC21F09FEC21F094
:1030E000000EF86E520EF76ED00EF66EB9EC21F0AF
:1030F000000EF86E520EF76EE60EF66EB9EC21F089
:1031000052EC20F09FEC21F055EC21F067C272F0F8
:1031100068C273F069C26FF06AC270F06BC274F07B
:103120006CC275F067C26AF068C26BF067C26CF07F
:1031300068C26DF06E6B69C260F06AC261F069C20C
:1031400062F06AC263F0646B6BC265F06CC266F0D9
:10315000696B6BC267F06CC268F067C278F068C2D6
:1031600079F069C276F06AC277F06BC27AF06CC20D
:103170007BF021EC01F0F1EC00F079EC01F001ECD6
:1031800001F0D1EC00F059EC01F011EC01F0E1ECB0
:1031900000F069EC01F0186A196A1A6A1B6A1C6A65
:1031A00018C030F219C031F21AC032F21BC033F22B
:1031B0001CC034F2C9EC36F032C02BF233C02CF212
:1031C00034C02DF235C02EF236C02FF22BC244F29D
:1031D0002CC245F22DC246F22EC247F22FC248F24F
:1031E00030C249F231C24AF232C24BF233C24CF21F
:1031F00034C24DF23F80AFEC1FF00A0E526E55EC18
:1032000021F00A0E516E0A0EA7EC21F02A0E3DB4F1
:10321000200EDBEC20F04A0EA7EC21F02A0E3DA494
:10322000200EDBEC20F03D7445EC20F071E29D6750
:1032300003D095EC03F03D98010E9D6303D0A0EC04
:1032400003F03D988EEC01F09E6703D04DEC03F047
:103250003D8A010E9E6303D07DEC03F03D9A020E81
:103260009E6303D022EC03F03D8A030E9E6303D0DD
:103270007DEC03F03D9A040E9E6303D06EEC03F0E8
:103280003D9A050E9E6303D05FEC03F03D9ABCECC3
:1032900001F0A66705D004EC03F0EAEC22F007D0B9
:1032A000010EA66304D0F4EC02F01FEC23F0A56736
:1032B00003D08AEC02F01DD0010EA56303D071EC9F
:1032C00002F017D0020EA56303D09AEC02F011D0E1
:1032D000030EA56303D0BAEC02F00BD0040EA56375
:1032E00003D0D6EC02F005D0050EA56302D0E5ECC4
:1032F00002F020EC23F082EC25F036EC26F0E7EC2F
:1033000021F05CEC20F0512E8FD7522E78D702D0CE
:10331000B6EC1FF0A2A502D08E6B8F6B89EC01F08A
:1033200082EC25F036EC26F0E7EC21F03F9012001D
:10333000140EA7EC21F052EF21F09CC045F09FEC59
:1033400021F0000EF86E530EF76E3E0EF66EB9ECDD
:1033500021F0000EF86E560EF76EAE0EF66EB9EC5A
:1033600021F055EC21F09C6710D0000EF86E530E42
:10337000F76E540EF66EB9EC21F0000EF86E530E97
:10338000F76E6A0EF66EB9EC21F0010E9C6310D058
:10339000000EF86E530EF76E800EF66EB9EC21F04B
:1033A000000EF86E530EF76E960EF66EB9EC21F025
:1033B000020E9C6310D0000EF86E530EF76EAC0E2A
:1033C000F66EB9EC21F0000EF86E530EF76EC20ED9
:1033D000F66EB9EC21F0ACDFF6EC07F00DE006E29A
:1033E0009C2B020E9C6501D09C6B05D09C079CAF6A
:1033F00002D0020E9C6FB5D745EC20F0EDE355EC02
:1034000021F0B9EC1FF0030E446006D0010E4462B7
:1034100003D048EC23F00ED045C09CF09FEC21F087
:10342000000EF86E510EF76E5C0EF66EB9EC21F0E0
:1034300050EC20F012009DC045F055EC21F09FECBF
:1034400021F0000EF86E540EF76E1A0EF66EB9ECFF
:1034500021F0000EF86E560EF76EAE0EF66EB9EC59
:1034600021F055EC21F09D6710D0000EF86E540E3F
:10347000F76E300EF66EB9EC21F0000EF86E540EB9
:10348000F76E460EF66EB9EC21F0010E9D6310D07A
:10349000000EF86E540EF76E5C0EF66EB9EC21F06D
:1034A000000EF86E540EF76E720EF66EB9EC21F047
:1034B0003FDFF6EC07F00DE006E29D2B010E9D6567
:1034C00001D09D6B05D09D079DAF02D0010E9D6F71
:1034D000C8D745EC20F0EDE355EC21F0B9EC1FF036
:1034E000030E446006D0010E446203D02DEC24F09C
:1034F0000ED045C09DF09FEC21F0000EF86E510EED
:10350000F76E5C0EF66EB9EC21F050EC20F0120074
:103510009EC045F09FEC21F0000EF86E540EF76E41
:10352000CA0EF66EB9EC21F0000EF86E560EF76E6C
:10353000AE0EF66EB9EC21F055EC21F09E6710D07E
:10354000000EF86E540EF76EE00EF66EB9EC21F038
:10355000000EF86E540EF76EF60EF66EB9EC21F012
:10356000010E9E6310D0000EF86E550EF76E0C0E15
:10357000F66EB9EC21F0000EF86E550EF76E220EC5
:10358000F66EB9EC21F0020E9E6310D0000EF86EBC
:10359000550EF76E380EF66EB9EC21F0000EF86E8F
:1035A000550EF76E4E0EF66EB9EC21F0030E9E63CB
:1035B00010D0000EF86E550EF76E640EF66EB9EC74
:1035C00021F0000EF86E540EF76E720EF66EB9EC26
:1035D00021F0040E9E6310D0000EF86E550EF76EAB
:1035E0007A0EF66EB9EC21F0000EF86E540EF76EFE
:1035F000720EF66EB9EC21F0050E9E6310D0000E2F
:10360000F86E550EF76E900EF66EB9EC21F0000EC6
:10361000F86E540EF76E720EF66EB9EC21F098EC5F
:1036200019F0F6EC07F00DE006E29E2B050E9E6504
:1036300001D09E6B05D09E079EAF02D0050E9E6FF7
:103640007BD745EC20F0EDE355EC21F0B9EC1FF011
:10365000030E44600AD0010E446207D02DEC24F022
:10366000020E9E6310D0C9EF16F045C09EF09FEC8D
:1036700021F0000EF86E510EF76E5C0EF66EB9EC8E
:1036800021F050EC20F01200A6C045F09FEC21F094
:10369000000EF86E550EF76EBC0EF66EB9EC21F00A
:1036A000000EF86E560EF76EAE0EF66EB9EC21F007
:1036B00055EC21F0A66710D0000EF86E540EF76E90
:1036C000300EF66EB9EC21F0000EF86E540EF76E67
:1036D000460EF66EB9EC21F0010EA66310D0000E76
:1036E000F86E540EF76E5C0EF66EB9EC21F0000E1B
:1036F000F86E540EF76E720EF66EB9EC21F098EC7F
:1037000019F0F6EC07F00DE006E2A62B010EA66517
:1037100001D0A66B05D0A607A6AF02D0010EA66FFA
:10372000C7D745EC20F0EBE355EC21F0B9EC1FF0E6
:10373000030E446006D0010E446203D08BEC23F0EC
:103740000ED045C0A6F09FEC21F0000EF86E510E91
:10375000F76E5C0EF66EB9EC21F050EC20F0120022
:10376000A5C045F09FEC21F0000EF86E550EF76EE7
:10377000E80EF66EB9EC21F0000EF86E560EF76EFC
:10378000AE0EF66EB9EC21F055EC21F0A56710D025
:10379000000EF86E540EF76EE00EF66EB9EC21F0E6
:1037A000000EF86E550EF76EFE0EF66EB9EC21F0B7
:1037B000010EA56310D0000EF86E550EF76E0C0EBC
:1037C000F66EB9EC21F0000EF86E560EF76E140E80
:1037D000F66EB9EC21F0020EA56310D0000EF86E63
:1037E000550EF76E380EF66EB9EC21F0000EF86E3D
:1037F000560EF76E2A0EF66EB9EC21F0030EA56395
:1038000010D0000EF86E550EF76E640EF66EB9EC21
:1038100021F0000EF86E540EF76E720EF66EB9ECD3
:1038200021F0040EA56310D0000EF86E550EF76E51
:103830007A0EF66EB9EC21F0000EF86E540EF76EAB
:10384000720EF66EB9EC21F0050EA56310D0000ED5
:10385000F86E550EF76E900EF66EB9EC21F0000E74
:10386000F86E540EF76E720EF66EB9EC21F098EC0D
:1038700019F0F6EC07F00DE006E2A52B050EA565A4
:1038800001D0A56B05D0A507A5AF02D0050EA56F89
:103890007BD745EC20F0EDE355EC21F0B9EC1FF0BF
:1038A000030E44600AD0010E446207D09DEC23F061
:1038B000020EA56310D023EF17F045C0A5F09FECD2
:1038C00021F0000EF86E510EF76E5C0EF66EB9EC3C
:1038D00021F050EC20F01200180EA7EC21F052EF6E
:1038E00021F09FC045F09FEC21F0A06713D0000E9F
:1038F000F86E5E0EF76E5C0EF66EB9EC21F0000EFF
:10390000F86E5E0EF76E9E0EF66EB9EC21F050EC7E
:1039100020F06ED055EC21F0000EF86E560EF76ECA
:10392000980EF66EB9EC21F0000EF86E560EF76E9A
:10393000AE0EF66EB9EC21F0010EA06308D0000EB9
:10394000F86E510EF76E3E0EF66EB9EC21F0020ED7
:10395000A06308D0000EF86E510EF76E380EF66EAA
:10396000B9EC21F041EC30F09FC018F0182A95EC2A
:103970003AF0010E376E74EC39F0000EF86E510E0D
:10398000F76E440EF66EBCEC21F0A6DFF6EC07F005
:1039900011E007E29F2B9F51A15DD8A401D09F6B3E
:1039A00006D09F079FAF03D0A1C09FF09F073BECBD
:1039B00022F0C2D745EC20F0E9E355EC21F0B9EC58
:1039C0001FF0030E446006D0010E446203D0E5EC04
:1039D00023F00ED045C09FF09FEC21F0000EF86E52
:1039E000510EF76E5C0EF66EB9EC21F050EC20F043
:1039F000120052EC21F05B0E3DAC590EA7EF21F006
:103A000055EC21F09C6716D0000EF86E500EF76E44
:103A1000580EF66EB9EC21F041EC30F06CC018F0A5
:103A20006DC019F095EC3AF0040E376E386A74ECFC
:103A300039F049D0010E9C6315D0000EF86E500E7F
:103A4000F76E460EF66EB9EC21F03AC24BF13BC26E
:103A50004CF13CC24DF13DC24EF13EC24FF11CEC67
:103A60003EF031D0020E9C632ED0000EF86E500E48
:103A7000F76E240EF66EB9EC21F03AC24BF13BC260
:103A80004CF13CC24DF13DC24EF13EC24FF107EC4C
:103A90003CF07CEC3CF05DEC00F013E3186A196A32
:103AA0001A6A1B6A1C6A18C050F119C051F11AC079
:103AB00052F11BC053F11CC054F1030E186E18C014
:103AC0005AF14CEC3EF03FA009D0000EF86E4F0EBC
:103AD000F76EEE0EF66EB9EC21F01CD0000EF86E0B
:103AE0004F0EF76EE80EF66EB9EC21F049C22DF0DC
:103AF0004AC22EF04BC22FF04CC230F04DC231F012
:103B0000ADEC3AF0040E376E020E386E4FEC3AF020
:103B1000A0EC39F03FB2F9EC1CF0120055EC21F0AA
:103B20009C6716D0000EF86E500EF76E600EF66EA3
:103B3000B9EC21F041EC30F062C018F063C019F02C
:103B400095EC3AF0040E376E386A74EC39F049D0CF
:103B5000010E9C6315D0000EF86E500EF76E4A0EE3
:103B6000F66EB9EC21F035C24BF136C24CF137C2DA
:103B70004DF138C24EF139C24FF11CEC3EF031D05C
:103B8000020E9C632ED0000EF86E500EF76E2A0EB9
:103B9000F66EB9EC21F03FC24BF140C24CF141C28C
:103BA0004DF142C24EF143C24FF107EC3CF07CECC8
:103BB0003CF05DEC00F013E3186A196A1A6A1B6A9C
:103BC0001C6A18C050F119C051F11AC052F11BC043
:103BD00053F11CC054F1030E186E18C05AF14CEC8E
:103BE0003EF03FA009D0000EF86E500EF76E180E92
:103BF000F66EB9EC21F024D0000EF86E4F0EF76E81
:103C0000FA0EF66EB9EC21F044C22DF045C22EF04A
:103C100046C22FF047C230F048C231F0ADEC3AF066
:103C2000030E376E010E386E4FEC3AF0A0EC39F00F
:103C3000000EF86E600EF76E5E0EF66EBCEC21F0B4
:103C40003FB2F9EC1CF01200A2A909D0000EF86EE8
:103C5000500EF76E0C0EF66EB9EC21F008D0000E87
:103C6000F86E500EF76E000EF66EB9EC21F01200F1
:103C700055EC21F09C6718D0000EF86E500EF76ED0
:103C8000680EF66EB9EC21F041EC30F067C018F028
:103C900068C019F095EC3AF0040E376E386A74EC8F
:103CA00039F024EC1EF008D1010E9C6317D0000EF1
:103CB000F86E500EF76E540EF66EB9EC21F03FC25E
:103CC0004BF140C24CF141C24DF142C24EF143C2F0
:103CD0004FF11CEC3EF024EC1EF0EED0020E9C6383
:103CE000EBD0A06709D0000EF86E510EF76E320EC1
:103CF000F66EB9EC21F029D0010EA06308D0000EB9
:103D0000F86E510EF76E3E0EF66EB9EC21F0020E13
:103D1000A06308D0000EF86E510EF76E380EF66EE6
:103D2000B9EC21F041EC30F09FC018F0182A95EC66
:103D30003AF0010E376E74EC39F0000EF86E510E49
:103D4000F76E440EF66EBCEC21F09D6708D0000EB5
:103D5000F86E500EF76ED20EF66EB9EC21F0010E31
:103D60009D6308D0000EF86E500EF76ED80EF66EFA
:103D7000B9EC21F09E6708D0000EF86E500EF76E79
:103D8000DE0EF66EB9EC21F0010E9E6308D0000E37
:103D9000F86E500EF76EE40EF66EB9EC21F0020EDE
:103DA0009E6308D0000EF86E500EF76EEA0EF66EA7
:103DB000B9EC21F0030E9E6308D0000EF86E500E91
:103DC000F76EF00EF66EB9EC21F0040E9E6308D08B
:103DD000000EF86E500EF76EF60EF66EB9EC21F08E
:103DE000050E9E6308D0000EF86E500EF76EFC0EA6
:103DF000F66EB9EC21F0A66708D0000EF86E510EF1
:103E0000F76E020EF66EB9EC21F0010EA66308D033
:103E1000000EF86E510EF76E080EF66EB9EC21F03A
:103E2000A56708D0000EF86E510EF76E0E0EF66EF6
:103E3000B9EC21F0010EA56308D0000EF86E510E0A
:103E4000F76E140EF66EB9EC21F0020EA56308D0E1
:103E5000000EF86E510EF76E1A0EF66EB9EC21F0E8
:103E6000030EA56308D0000EF86E510EF76E200EFB
:103E7000F66EB9EC21F0040EA56308D0000EF86EC2
:103E8000510EF76E260EF66EB9EC21F0050EA56305
:103E900008D0000EF86E510EF76E2C0EF66EB9ECCF
:103EA00021F0020E9C6308D01A0EA7EC21F0200E20
:103EB000A2B9240EDBEC20F03FB2F9EC1CF01200AA
:103EC00055EC21F0000EF86E500EF76E380EF66EBF
:103ED000B9EC21F062C22DF063C22EF064C22FF063
:103EE00065C230F066C231F032D806EC35F080ECB5
:103EF00030F0ADEC3AF0030E376E010E386E4FEC39
:103F00003AF0A0EC39F0000EF86E500EF76E3E0E4F
:103F1000F66EBCEC21F00EC14BF10FC14CF110C19B
:103F20004DF111C14EF112C14FF107EC3CF07CECA8
:103F30003CF0F9EC3EF0000EF86E500EF76E440EB9
:103F4000F66EBCEC21F03FB2F9EC1CF01200410E11
:103F5000366E880E356E326A336A346A120050DD6E
:103F6000DDDD86DEADD791D8FEE312008ED8FEE20D
:103F70001200F9DF446A60EC20F081B603D0010E34
:103F8000446E05D081B403D0020E446E00D00A0EF8
:103F90004F6E5CEC20F045EC20F076E34F2EF9D725
:103FA0000A0E44269FEC21F03DB026D00B0E446251
:103FB0002CD0A76709D0000EF86E510EF76E520E86
:103FC000F66EB9EC21F05BD0010EA76309D0000EAC
:103FD000F86E510EF76E5C0EF66EB9EC21F04FD014
:103FE000020EA76309D0000EF86E510EF76E680E30
:103FF000F66EB9EC21F043D0000EF86E510EF76E5C
:10400000460EF66EB9EC21F03AD03EBC30D00C0E24
:1040100044622CD055EC21F0000EF86E510EF76E74
:10402000740EF66EB9EC21F0A279A2B909D0000E97
:10403000F86E510EF76E8A0EF66EB9EC21F008D0CC
:10404000000EF86E510EF76E9C0EF66EB9EC21F074
:104050006BEC23F072EC23F04FEC23F041EC23F0F7
:1040600033EC23F03BEC22F0F5EC24F008D0000E0A
:10407000F86E510EF76E5C0EF66EB9EC21F0B6ECF0
:104080001FF09FEC21F03D821200040081B601D0A8
:1040900005D081B401D002D0D8901200D88012008F
:1040A00052EC20F058EC20F058EC20F058EC20F0C6
:1040B000FA0E09D0C80E07D0640E05D0320E03D018
:1040C0000A0E01D0010E0400426EC80E406E150E9D
:1040D000416E402EFED7412EFCD7422EF6D712005D
:1040E0008B908B968B94EADF300EF0D8EBDF300E9E
:1040F000EDD8E8DF300EEAD8E5DF200EE7D8E0DFC4
:10410000290ED4D8080ED2D8060ED0D8010ECED89B
:10411000020ECCD80C0ECAD876D8C7D055EC21F0F8
:104120000ED9000EF86E5F0EF76E9E0EF66EB9ECAD
:1041300021F0000EF86E5F0EF76EB40EF66EB9EC5D
:1041400021F0000EF86E5F0EF76ECA0EF66EB9EC37
:1041500021F0000EF86E600EF76E0C0EF66EB9ECE4
:1041600021F0120055EC21F0EAD8000EF86E5F0E37
:10417000F76E9E0EF66EB9EC21F0000EF86E5F0E33
:10418000F76EB40EF66EB9EC21F0000EF86E5F0E0D
:10419000F76EE00EF66EB9EC21F0000EF86E5F0ED1
:1041A000F76EF60EF66EB9EC21F01200000000007A
:1041B000000000001200086E9BD808508B86D6ECD9
:1041C00020F08B94D6EC20F08B90D6EC20F0F00B06
:1041D0007DD80838F00B7AD0086E084608460846A5
:1041E00087D80850400962D8080E4F6E0900F55074
:1041F000E2DF4F2EFBD71200000EF86E420EF76E74
:10420000640EF66E06D0000EF86E420EF76E240EA7
:10421000F66E080E506E516A5150DEDF512A502E54
:10422000FBD7120000001818181B000000001B1B11
:104230001B1B000000000303031B00000E110E00F7
:10424000001F00000E110E000D1513000E110E00C0
:104250000A1515000E110E021F0A060000000000CC
:10426000001B00001F1F1F1F1F1F1F1F001F1F1FDE
:104270001F1F1F1F00001F1F1F1F1F1F0000001FE9
:104280001F1F1F1F000000001F1F1F1F0000000036
:10429000001F1F1F0000000000001F1F0000000083
:1042A0000000001FB5C0E8FF01D00C0E086E20D83A
:1042B0000850F00B8B96D6EC20F08B94D6EC20F0C7
:1042C0008B90D6EC20F002D80838F00B040082B0B6
:1042D000010982B2020982B4040982B60809826E19
:1042E000D6EC20F08B80D6EC20F08B90D6EF20F02F
:1042F0000400828ED6EC20F0948ED6EC20F08B96C3
:10430000D6EC20F08B845368534E15D0D6EC20F0B9
:104310003A96D6EC20F08B80D6EC20F082AE3A862E
:10432000D6EC20F08B90D6EC20F08B80D6EC20F0F1
:104330008B903AA6E9D7949E8B94D6EF20F0010E8D
:10434000B5DF020EB3D7800EB1D7C00EAFD780094C
:10435000ADD7200E30D74F6EFCDF4F2EFDD71200A9
:10436000096E09380EEC00F026DF09500EEC00F063
:1043700022D70900F550EBDF0900F55002E01BDF02
:10438000FBD71200140E526E010E5B6E100E5D6EA6
:104390003D84CEEC21F0150E526E3D94E7EC21F0F9
:1043A00060EC20F060EC20F0D8803DA4D8905B3623
:1043B0005C365D365E365F365D883DA45D98522E74
:1043C000EDD712005B6A5C6A5D6A5E6A5F6A050E21
:1043D0004F6E506A00EE5BF050C05AF0502AEE501B
:1043E000F5EC21F04F2EF8D712008C6E5A6602D0F1
:1043F000898C17D0010E5A6202D0898E12D0020E1B
:104400005A6202D08D840DD0030E5A6202D08D8282
:1044100008D0040E5A6201D08D80050E5A6201D078
:10442000898A899C899E8D908D928D94899A12009B
:1044300045689F6701D04590010E9F6301D045926A
:10444000020E9F6301D04594030E9F6301D04596F1
:10445000040E9F6301D04598050E9F6301D0459AD5
:10446000060E9F6301D0459C459EA2B9458E050E60
:104470005A6E4550BAD7A2BD01D001D0D9D7456AEE
:104480009F6701D04580010E9F6301D04582020ED7
:104490009F6301D04584030E9F6301D04586040EBF
:1044A0009F6301D04588050E9F6301D0458A060EA3
:1044B0009F6301D0458CA2B9458E050E5A6E4550BA
:1044C00094D7F00ED36E400E9B6E0F01806A896AFE
:1044D000070E386F0F0E926E816A8A6A000E396F6E
:1044E0000F0E936E826A8B6A000E946E000E3A6F06
:1044F000836A8C6A000E956E000E3B6F846A8D6A2B
:10450000000E3C6F000E966E040EC16EBE0EC06EA5
:10451000000ED06EF00EF26E000EF16E000EF06E18
:10452000010E9D6E000EA06E000EA36E310ECD6EBC
:10453000000EBA6E000EB16EB10ECF6EE00ECE6EF2
:10454000310ECD6E010E9D6E000EA06E4D0ED66E1C
:10455000070ED56EF60ED76E3C0ED66E0001120019
:104560004F6A00EE00F0EE6A4F2EFDD7040E506E3B
:1045700001EE00F0EE6A4F2EFDD7502EFBD7120051
:1045800011EC22F0E2EF21F014DA01DA24DA79D822
:1045900080D969D822D90FD9FCD82FDAB2D8C3D89C
:1045A000D4D899D89FD87BD8E2D83BEC22F037DA20
:1045B00048DA25EC00F033EF00F0FF0EBB6E0C0E76
:1045C000666E976B986B3CD8000EBA6E030EBC6E8D
:1045D000BA841200A2BB05D093C091F094C092F0AF
:1045E0002CD09651945D02E19551935DD8A401D0F1
:1045F00007D09451965D02E19351955DD8B007D0F4
:10460000640E866F93C095F094C096F012D08667C2
:1046100015D0876713D0140E186E000E196E18503F
:10462000955F1950965B0A0E876F96AF02D0956B17
:10463000966B95C091F096C092F001D812001200CE
:1046400097C04FF098C050F0D89050324F32D89069
:1046500050324F324FC067FF6698669A97B16688AE
:1046600097B3668A1200A2A9FFEC23F0A2B911EC5D
:1046700024F01200A2A9F7EC23F0A2B909EC24F06F
:104680001200A2A935EC24F0A2B93FEC24F01200EC
:10469000A2A91BEC24F0A2B923EC24F01200A2A9D9
:1046A000A3EC24F0A2B9B5EC24F01200A2A99BEC73
:1046B00024F0A2B9ADEC24F01200A2A953EC24F02E
:1046C000A2B977EC24F01200A2A965EC24F0A2B9FB
:1046D00089EC24F01200A2A95BEC24F0A2B97FECD3
:1046E00024F01200A2A96DEC24F0A2B991EC24F000
:1046F0001200480E066E020E4F6E00EEA3F03FEF62
:1047000025F0480E066E020E4F6E00EEA3F053EC3D
:1047100025F05AEF20F04B0E066E010E4F6E00EEA4
:10472000A6F03FEF25F04B0E066E010E4F6E00EE29
:10473000A6F053EC25F05AEF20F0110E066E010E94
:104740004F6E00EEA5F03FEF25F0110E066E010E44
:104750004F6E00EEA5F053EC25F05AEF20F04E0E10
:10476000066E010E4F6E00EEB5F03FEF25F04E0ED7
:10477000066E010E4F6E00EEB5F053EC25F05AEFC9
:1047800020F0100E066E010E4F6E00EEA1F03FEF0E
:1047900025F0100E066E010E4F6E00EEA1F053ECE8
:1047A00025F05AEF20F00F0E066E010E4F6E00EE50
:1047B000A0F03FEF25F00F0E066E010E4F6E00EEDB
:1047C000A0F053EC25F05AEF20F00E0E066E010E0D
:1047D0004F6E00EE9FF03FEF25F00E0E066E010EBD
:1047E0004F6E00EE9FF053EC25F05AEF20F0120EC2
:1047F000066E050E4F6E02EE62F03FEF25F0120ED0
:10480000066E050E4F6E02EE62F053EC25F05AEF85
:1048100020F0170E066E050E4F6E02EE62F03FEFAF
:1048200025F0170E066E050E4F6E02EE62F053EC89
:1048300025F05AEF20F0050E066E010E4F6E00EEC9
:104840009CF03FEF25F00B0E066E010E4F6E00EE52
:104850009CF03FEC25F05AEF20F00C0E066E020E95
:104860004F6E00EE9DF03FEF25F0050E066E010E37
:104870004F6E00EE9CF053EC25F05AEF20F00B0E3B
:10488000066E010E4F6E00EE9CF053EC25F05AEFD1
:1048900020F00C0E066E020E4F6E00EE9DF053ECF3
:1048A00025F05AEF20F01C0E066E0A0E4F6E02EE37
:1048B00008F03FEF25F01C0E066E0A0E4F6E02EE5A
:1048C00008F053EC25F05AEF20F0260E066E0A0E83
:1048D0004F6E02EE12F03FEF25F0260E066E0A0E26
:1048E0004F6E02EE12F053EC25F05AEF20F0300E2E
:1048F000066E0A0E4F6E02EE08F03FEF25F0300E06
:10490000066E0A0E4F6E02EE08F053EC25F05AEFD9
:1049100020F03A0E066E0A0E4F6E02EE12F03FEFD6
:1049200025F03A0E066E0A0E4F6E02EE12F053ECB0
:1049300025F05AEF20F0000E066E050E4F6E02EEC7
:104940005DF03FEF25F0000E066E050E4F6E02EE95
:104950005DF053EC25F05AEF20F0060E066E050EC2
:104960004F6E02EE5DF03FEF25F0060E066E050E6F
:104970004F6E02EE5DF053EC25F05AEF20F04A0E38
:10498000066E010E4F6E02EE02F03FEF25F04A0E6A
:10499000066E010E4F6E02EE02F053EC25F05AEF58
:1049A00020F0440E066E020E4F6E02EE00F03FEF56
:1049B00025F0440E066E020E4F6E02EE00F053EC30
:1049C00025F05AEF20F0460E066E020E4F6E02EEF4
:1049D00003F03FEF25F0460E066E020E4F6E02EE1C
:1049E00003F053EC25F05AEF20F0470E066E010E4F
:1049F0004F6E00EEA2F03FEF25F0470E066E010E5F
:104A00004F6E00EEA2F053EC25F05AEF20F04C0E62
:104A1000066E010E4F6E02EE81F03FEF25F04C0E58
:104A2000066E010E4F6E02EE81F053EC25F05AEF48
:104A300020F04D0E066E010E4F6E02EE82F03FEF3B
:104A400025F04D0E066E010E4F6E02EE82F053EC15
:104A500025F05AEF20F0A6B2FED706C0A9FF07C086
:104A6000A8FFA69EA69CA684F29EF2BEFED7550E77
:104A7000A76EAA0EA76EA682F28EA694120004005C
:104A8000EECF07F02BEC25F0062A4F2EF8D74DEF8E
:104A900018F0A6B2FED706C0A9FFA69EA69CA680C7
:104AA000A850076E1200040049EC25F007C0EEFF85
:104AB000062A4F2EF8D712001D0E0DD0190E0BD05E
:104AC000150E09D0110E07D00D0E05D0090E03D01A
:104AD000050E01D0010EC26EC282C2B2FED7C4CF93
:104AE00055F0C3CF54F012005B6A5C6A5D905D9232
:104AF0005D945D9612005E6A5F6A5D985D9A5D9C4A
:104B00005D9E12003DA814D0A2A70BD074EC25F036
:104B10007EC018F0A3EC25F07CC018F0A3EC25F0C3
:104B200011D074EC25F07CC018F0A3EC25F00AD06D
:104B300074EC25F07CC018F0F8EC25F07EC018F07D
:104B4000A3EC25F01200150E1D6E18501D5E1D2ED3
:104B500002D05D8612001D2E02D05D8412001D2E33
:104B600002D05D8212001D2E02D05D8012001D2E2B
:104B700002D05C8E12001D2E02D05C8C12001D2E05
:104B800002D05C8A12001D2E02D05C8812001D2EFD
:104B900002D05C8612001D2E02D05C8412001D2EF5
:104BA00002D05C8212001D2E02D05C8012001D2EED
:104BB00002D05B8E12001D2E02D05B8C12001D2EC7
:104BC00002D05B8A12001D2E02D05B8812001D2EBF
:104BD00002D05B8612001D2E02D05B8412001D2EB7
:104BE00002D05B8212001D2E02D05B8012001200E8
:104BF000182A184E12005B80184E12005B82184E65
:104C000012005B84184E12005B86184E12005B88FF
:104C1000184E12005B8A184E12005B8C184E120060
:104C20005B8E184E12005C80184E12005C82184E8B
:104C300012005C84184E12005C86184E12005C88CC
:104C4000184E12005C8A184E12005C8C184E12002E
:104C50005C8E184E12005D80184E12005D82184E58
:104C600012005D84184E12005D8612003DAA14D019
:104C7000A2A70BD07BEC25F081C018F057EC26F0F2
:104C80007FC018F057EC26F011D07BEC25F07FC0E8
:104C900018F057EC26F00AD07BEC25F07FC018F016
:104CA000ACEC26F081C018F057EC26F01200150E7F
:104CB0001D6E18501D5E1D2E02D05F8E12001D2E1F
:104CC00002D05F8C12001D2E02D05F8A12001D2EB2
:104CD00002D05F8812001D2E02D05F8612001D2EAA
:104CE00002D05F8412001D2E02D05F8212001D2EA2
:104CF00002D05F8012001D2E02D05E8E12001D2E8B
:104D000002D05E8C12001D2E02D05E8A12001D2E73
:104D100002D05E8812001D2E02D05E8612001D2E6B
:104D200002D05E8412001D2E02D05E8212001D2E63
:104D300002D05E8012001D2E02D05D8E12001D2E4C
:104D400002D05D8C12001D2E02D05D8A12001D2E35
:104D500002D05D8812001200182A184E12005D88D9
:104D6000184E12005D8A184E12005D8C184E12000B
:104D70005D8E184E12005E80184E12005E82184E34
:104D800012005E84184E12005E86184E12005E8875
:104D9000184E12005E8A184E12005E8C184E1200D9
:104DA0005E8E184E12005F80184E12005F82184E01
:104DB00012005F84184E12005F86184E12005F8842
:104DC000184E12005F8A184E12005F8C184E1200A7
:104DD0005F8E1200140E4F6E03EE00F081CFE8FFDD
:104DE000120BE8CFEEFFD6EC20F04F2EF7D70DD008
:104DF000140E4F6E03EE00F081CFE8FF030BE8CFF7
:104E0000EEFFD6EC20F04F2EF7D7AA6BAB6BAC6B56
:104E1000AD6BAE6BAF6BB06BB16BB26BB36B130EB4
:104E20004F6E03EE00F0EECFAAF0EECFB3F0B26714
:104E30000AD0B3C0E8FFAA5D02E1AB2B27D0B22BAA
:104E4000B3C0ACF023D0010EB2630AD0B3C0E8FF08
:104E5000AC5D02E1AD2B1AD0B22BB3C0AEF016D0D0
:104E6000020EB2630AD0B3C0E8FFAE5D02E1AF2B21
:104E70000DD0B22BB3C0B0F009D0030EB26306D090
:104E8000B3C0E8FFB05D02E1B12B00D04F2ECDD70B
:104E9000ABC0B2F0AAC0A9F0AD51B25DD8B004D099
:104EA000ADC0B2F0ACC0A9F0AF51B25DD8B004D083
:104EB000AFC0B2F0AEC0A9F0B151B25DD8B004D06D
:104EC000B1C0B2F0B0C0A9F01200006ED8CF01F0AE
:104ED000E0CF02F09EA034D09E9082678207836765
:104EE00083078467840785678507866786078767E2
:104EF0008707886702D0895306E088078829D8B4D5
:104F00008907D8B488538D678D078C678C078A67AB
:104F100002D08B5306E08A078A29D8B48B07D8B40D
:104F20008A538E6702D08F5306E08E078E29D8B43D
:104F30008F07D8B48E53B10ECF6EE00ECE6E26D052
:104F4000F2A21AD0F292F298D58EF8EC26F0A2B323
:104F5000596CA2A103D0F17CF1AC06D0A9A302D078
:104F6000592A07D0590605D0A9B302D0592A01D031
:104F70005906A2B3596C0AD0F2A408D0F294F28870
:104F8000D59EF60ED76E3C0ED66E00D002C0E0FF66
:104F9000005001C0D8FF1000036ED8CF04F0E0CF5E
:104FA00005F005C0E0FF035004C0D8FF1000540E08
:104FB00005D0140E03D0400E01D0000EA7EC21F056
:104FC000000EF86E4F0EF76ED20EF66EBCEC21F0AE
:104FD00012002020202020202020202020202020FF
:104FE00020202020202000000B5357523D000B535F
:104FF00057523D202D2C2D2D00004B524C3D0000D2
:105000001F4D657373482E20312000001F4D6573BE
:1050100073482E20322000004B524C3D202D2C2D69
:10502000644200000050703D00004050723D00009E
:105030004D5B5365635D0000544C45443D00644244
:105040006D205B005D0000503D0040463D00145067
:10505000663D000014523D0000414443703D000095
:1050600040414443663D000014414443723D00000A
:10507000002D2D2D2D2D20414443203064426D20E4
:105080002D2D2D2D2D00002D2D2D2D204144432083
:105090002D333064426D202D2D2D2D004041444391
:1050A00020203064426D3A00144144432D33306473
:1050B000426D3A004056616C2E3A0000144B6579FF
:1050C000526F746174653D537465702020202020F8
:1050D00020001B5B50702C001B5B50662C001F5285
:1050E0004C2C00001F52692C00001F53572C00004D
:1050F0001F50722C00001F31302C00001F32302C4A
:1051000000002250702C00002250662C0000255216
:105110004C5D00002552695D00002553575D00007D
:105120002550725D00002531305D00002532305D74
:105130000000144D6F64650014416E745B001454DC
:1051400052585B005D00004B6579206C6F6E6720E4
:1051500020000053455455502D3E00000041424F61
:10516000525420202D3E0000004368616E67652088
:105170002D3E0000006D65617375722E6865616477
:105180002D6368616E67652D3E00406D65617375C6
:1051900072696E672068656164203100406D6561E9
:1051A000737572696E672068656164203200004122
:1051B000444355666F72772E3A004041444355662A
:1051C000504550203A0000414443557265742E20EA
:1051D0003A00144C6576656C313A203064426D209B
:1051E0002020202020202000144C6576656C323A67
:1051F000202D333064426D20202020202000003DEF
:105200003D2041443833303720466F7277617264F5
:10521000203D3D00003D3D20414438333037205291
:10522000657475726E20203D3D00406D6B783A00CC
:10523000146D6B793A005473686F72743D4F4B2054
:105240006C6F6E673D41626F727420005473686FBB
:1052500072743D4F4B206C6F6E673D4368616E67A3
:105260006500544B6579202D3E206E6578742020B2
:105270002020202020202000003D3D3D3D3D3D20C0
:105280004D656E7565203D3D3D3D3D3D3D00405BBE
:10529000315D5265747269657665204D617820765E
:1052A000616C2E001420206F6620746865206C618C
:1052B00073742078206D696E2E0054202041626F37
:1052C0007274204B65792D6C6F6E67202020200052
:1052D000003D205265747269657665204D617820C5
:1052E00076616C2E3D001445786974207769746886
:1052F000204B65792120202020202000405B325D5A
:10530000204C4344204D6F646520446973706C6188
:10531000790014202020204144432C2064426D2039
:10532000616E6420202020005420202020506F77C0
:105330006572202020202020202020200000003D19
:10534000204C4344204D6F646520446973706C6148
:1053500079203D00143020446973706C61792069B4
:105360006E20414443202020200054202041442D21
:10537000436F6E7665727465722078203820200045
:10538000143120446973706C617920696E20644225
:105390006D202020200054202020202020202020AC
:1053A00020202020202020202020200014322044F3
:1053B0006973706C617920696E20506F7765722C0B
:1053C000200054202053575220616E64205265748F
:1053D00075726E4C6F737300405B335D204C4544B7
:1053E0002042617231206C656674202020001420F8
:1053F00020202050455020616E642050666F7277E7
:1054000061726400542020202020202020202020B1
:1054100020202020202020202000003D3D204C4541
:10542000442042617231206C65667420203D3D004D
:10543000143020506F776572205045502020202076
:10544000202020202000542020456E76656C6F704F
:1054500070652067726561746520200014312050EA
:105460006F77657220466F7277617264202020200A
:1054700020005420617070726F78696D61746520CE
:105480006176657261676500405B345D204C454420
:1054900020426172322072696768742020001420F3
:1054A000526574204C6F73732C20524C6F737320B1
:1054B000696E760054205357522C2050722C205085
:1054C000722B31302F3230644200003D3D204C457C
:1054D00044204261723220726967687420203D0066
:1054E00014302052657475726E204C6F73732028CF
:1054F0006462292020005420204C454420302E2E68
:10550000323020302E2E34306442200014312052AC
:105510004C6F737320696E766572732028646229FC
:1055200020005420204C454420302E2E3230203490
:10553000302E2E3064422000143220535752203136
:105540002C3020746F20782C7820202020005420CC
:10555000204C454420302E2E323020312C302E2E3F
:10556000782C7800143320506F7765722052657460
:1055700075726E2020202020200014342050726587
:105580007475726E202B3130644220202020200060
:105590001435205072657475726E202B323064425F
:1055A000202020202000405B355D2050574D312DBC
:1055B0004F7574707574202020202000003D3D3D03
:1055C0002050574D31204F7574707574203D3D3D0E
:1055D0003D00405B365D2050574D322D4F75747045
:1055E0007574202020202000003D3D3D2050574D67
:1055F00032204F757470757420203D3D3D0054205D
:10560000302E2E34306442202D3E20302E2E355642
:105610006F6C740054202034302E2E306442202DC4
:105620003E20302E2E3556202000542020312E30A2
:105630002E2E782E78202D3E20302E2E355620000E
:10564000405B375D20545258204368616E6E656C34
:105650002020202020001420202020776869636803
:1056600020737769746368657320200054202020BC
:105670002072656C617973207468726F7567682039
:105680002000405B375D20416E74656E6E61204E78
:10569000756D626572732000003D3D2073776974FB
:1056A00063682052656C616973203D3D3D00403D5B
:1056B0003D3D3D3D3D3D3D3D3D3D3D3D3D3D3D3D1A
:1056C0003D3D3D00003D3D3D3D3D3D205345545554
:1056D00050203D3D3D3D3D3D3D00405B305D204126
:1056E000626F7274202020202020202020202000A3
:1056F000405B315D2055666F72772E2063616C6967
:1057000062726174650014202020206D65617375DC
:1057100072696E6720686561642020005420202033
:1057200020414438333037202831292020202020C0
:105730002000405B325D205572657475726E206387
:10574000616C6962722E2000542020202041443870
:105750003330372028322920202020202000405BB1
:10576000335D2064697265632E20436F75706C65CC
:10577000722020001420202020636F75706C696EE9
:1057800067206C6F73732020200054202020207726
:10579000696E64696E6720737465656C20202000F3
:1057A000002D2064697265632E436F75706C65729D
:1057B0004D4831202D00002D2064697265632E4311
:1057C0006F75706C65724D4832202D004020436F1C
:1057D00075706C696E67206C6F73732020202020B9
:1057E0002000145764673A001E3D0000405B345DA2
:1057F000204C434420446973706C61792054696D76
:105800006500142020202056616C7565205045509D
:105810002020202020202000542020202050722CE6
:105820002053575220756E6420524C202000002DCA
:10583000204C434420446973706C61792054696D35
:1058400065202D00405B355D204C4544204261724F
:1058500067726170682020202000142020202050D2
:1058600065616B26486F6C642054696D652020006B
:105870005420202020616E6420506F696E74264889
:105880006F6C64202000002D2D2D204C45442042BB
:1058900061726772617068202D2D2D00405B365D4E
:1058A0002056696577204D6B2E686561642D666FA3
:1058B00072001420202020414443312C3220616E9C
:1058C00064206D6B7820200054202020206D6B799F
:1058D0002056616C75652020202020202000405B30
:1058E000375D2056696577204D2E686561642D62AD
:1058F00061636B00405B385D2052656C6169732D9C
:105900004D6F64652020202020001420202020548A
:1059100052582C20416E74656E6E65202020200048
:1059200054202020206F7220776974686F7574206E
:1059300052656C2E2000002052656C61792D436FFA
:105940006E74726F6C20202020202000402D2D2DA1
:105950002D2D2D2053656C656374202D2D2D2D2D3F
:105960002D00145B305D20776974686F7574205268
:10597000656C616973202000145B315D20545258BE
:105980002053776974636820202020202000145B56
:10599000325D20416E74656E6E6173205377697459
:1059A00063682000405B395D2052656C6179206E30
:1059B000756D626572206F662000142020202041E2
:1059C000637475616C2072656C61797320202000AE
:1059D0005420202020202020202020202020202093
:1059E000202020202000002D2052656C6169732D3D
:1059F0006E756D626572206F66202D00402D2D2D15
:105A00002D2D2D204D6178696D756D202D2D2D2D3D
:105A10002D001452656C6169733A0000405B3130AF
:105A20005D204C45442F50574D20636865636B20C3
:105A3000200014202020204C454420426172672E13
:105A400020312F32202020005420202020616E643D
:105A50002050574D20312F32202020202000002DB3
:105A60002D2D204C45442F50574D20636865636BA6
:105A7000202D2D00402D2D2D207769746820726F08
:105A80007461727920456E632E00144C612F623A66
:105A900000001E50574D3A00405B31315D20526F7F
:105AA000742E656E632E54797065202020001420BA
:105AB00020646966666572656E74207479706573BA
:105AC000202020005420646972656374696F6E2021
:105AD0006F6620726F7461742E00002D2D2D205280
:105AE0006F742E656E632E54797065202D2D2D00F8
:105AF000405261737420322C205374657031205BE6
:105B0000000014526576657273202020202020202A
:105B1000205B0000405B31325D204D61782E636177
:105B20002E2D6F66662076616C0014202073746FD2
:105B3000726167652074696D6520616E6420200064
:105B40005420204C434420434C52206F6E2F6F66EC
:105B50006620202020000020534554204D61782EDF
:105B600063612E2D6F66662076616C0040686F6CF5
:105B7000642074696D653A0014566965772074680D
:105B8000656E20434C52205B0000405B31335D204A
:105B90004D616E75656C6C204D4B666F72772000A1
:105BA00014202063616C6962726174652077697486
:105BB000686F7574200054202052462D47656E652D
:105BC0007261746F7220202020202000405B3134ED
:105BD0005D204D616E75656C6C204D4B6261636B31
:105BE0002000405B31355D2050574D205365747463
:105BF000696E677320202000142020706F696E7416
:105C0000657220696E6572746961202020005420DD
:105C100020504550205065616B26486F6C642020F1
:105C200020202000002D2D2D2050574D205365742D
:105C300074696E6773202D2D2D004054696D657257
:105C4000503A0000145045502C5065616B26486F47
:105C50002E206C6F6E675B00405B31365D205357C2
:105C6000522D446973706C61792D4C4544001420A9
:105C70002053657474696E67207468652020202045
:105C800020202000542020646973706C6179207298
:105C9000616E6765202020202000002D2D205357A5
:105CA000562D446973706C61792D4C4544202D004C
:105CB000405B31375D205357522D446973706C61DE
:105CC000792D50574D00002D2D205357522D4469EA
:105CD00073706C61792D50574D202D00405B313829
:105CE0005D2052656C61697320696E766572732000
:105CF0002000002D2D2052656C61697320696E763D
:105D0000657273202D2D2D0014202052656C616961
:105D10007320696E76657273202020202000542045
:105D200020737769746368204F4E2F4F46462020BA
:105D3000202020004052656C61697320696E766591
:105D40007273205B0000405B31395D205049432D68
:105D50005761746368646F6720202000002D2D2D2B
:105D6000205049432D5761746368646F67202D2D5F
:105D70002D001420205265737461727473202020EA
:105D80002020202020202000542020636F756E7476
:105D90006564212120202020202020202000405246
:105DA000657374617274733A0000405B32305D2039
:105DB000437572736F722074797065202020200003
:105DC00014202054797065206F6620636F7572739C
:105DD00065202020200054202073657420757021D8
:105DE000212020202020202020202000002D2043C2
:105DF0007572736F7220534554202D2D2D2D2D2D2E
:105E0000200040437572736F722D3E414243000083
:105E100040437572736F722D3E00003D3D3D3D2045
:105E2000536176652044617461203D3D3D3D3D00F8
:105E3000403D3D3D3D3D3D3D20746F203D3D3D3D60
:105E40003D3D3D3D3D00143D3D3D3D2050494320FD
:105E5000456570726F6D203D3D3D3D00003D3D3D0F
:105E60003D3D2046756E6374696F6E203D3D3D3D3E
:105E70003D00402D2D2D2D2D2D2041626F7274205F
:105E80002121202D2D2D2D00143D3D3D3D3D3D3D3D
:105E90003D3D3D3D3D3D3D3D3D3D3D3D3D00403D6C
:105EA0003D3D3D3D206465616374697665203D3DFF
:105EB0003D3D3D00003D3D3D3D20526566657265BE
:105EC0006E6365203D3D3D3D3D00402020506C65AA
:105ED000617365206E6F746520616E642020200000
:105EE0001420617263686976652074686520666F46
:105EF0006C6C6F772E005420203220414443207672
:105F0000616C756573212120202020000073746569
:105F1000702077696474682031302020000000739D
:105F200074657020776964746820312020004020F7
:105F30002028302C3520626973203130205365636E
:105F400029202000144C434468616E673A001453C2
:105F5000575220312C302062697320004020535763
:105F6000522D52616E6765202020202020202020A5
:105F70002000405065616B2D4C45443A00001450A0
:105F80006F696E742D5065616B202020205B0000CE
:105F90006D5365630000536563004D696E00003DFD
:105FA0003D20576174742D5357522D4D65746572A1
:105FB000203D3D00403D20316D5720757020746FAD
:105FC000203135303057203D3D00143D3D3D3D20D2
:105FD00028632920444C344A414C203D3D3D3D003E
:105FE000143D2048573A2056657273696F6E203110
:105FF0002E3031203D00543D3D2053573A20566508
:1060000072732E20312E3138203D3D00543D3D3DF0
:106010003D2032342E30322E32303231203D3D3D63
:106020003D002D2D2D00494E46006D57000075573F
:1060300000006E570000705700006657000061575F
:106040000000572000006B570000205600006D56DE
:106050000000755600006E56000064426D006442F8
:1060600000007373000013D806D8136A146A156A07
:10607000166A176A12000E6A0F6A106A116A126AAB
:106080001200186A196A1A6A1B6A1C6A1200F9DF80
:106090001D6A1E6A1F6A206A216A12002D6A2E6A12
:1060A0002F6A306A316A12000EC132F00FC133F02C
:1060B00010C134F011C135F012C136F012000EC11A
:1060C0002DF00FC12EF010C12FF011C130F012C110
:1060D00031F0120032C02DF033C02EF034C02FF05A
:1060E00035C030F036C031F012002DC032F02EC075
:1060F00033F02FC034F030C035F031C036F012002C
:106100002DC00EF12EC00FF12FC010F130C011F1D3
:1061100031C012F1120013C12DF014C12EF015C1BF
:106120002FF016C130F017C131F0120013C132F058
:1061300014C133F015C134F016C135F017C136F073
:10614000120018C12DF019C12EF01AC12FF01BC179
:1061500030F01CC131F0120018C132F019C133F017
:106160001AC134F01BC135F01CC136F012001DC13C
:106170002DF01EC12EF01FC12FF020C130F021C123
:1061800031F012001DC132F01EC133F01FC134F0D6
:1061900020C135F021C136F0120022C12DF023C1FB
:1061A0002EF024C12FF025C130F026C131F01200AD
:1061B00022C132F023C133F024C134F025C135F0BF
:1061C00026C136F0120027C12DF028C12EF029C1BA
:1061D0002FF02AC130F02BC131F0120027C132F06C
:1061E00028C133F029C134F02AC135F02BC136F073
:1061F000120032C013F133C014F134C015F135C0B0
:1062000016F136C017F112002DC013F12EC014F193
:106210002FC015F130C016F131C017F112002DC09A
:1062200018F12EC019F12FC01AF130C01BF131C086
:106230001CF112002DC01DF12EC01EF12FC01FF148
:1062400030C020F131C021F112002DC022F12EC04A
:1062500023F12FC024F130C025F131C026F1120006
:106260002DC027F12EC028F12FC029F130C02AF10E
:1062700031C02BF112000EC018F00FC019F010C081
:106280001AF011C01BF012C01CF012000EC01DF05D
:106290000FC01EF010C01FF011C020F012C021F07E
:1062A000120018C00EF019C00FF01AC010F01BC079
:1062B00011F01CC012F012001D361E361F3620369B
:1062C00021361200183619361A361B361C361200C3
:1062D000213220321F321E321D3212001C321B327C
:1062E0001A3219321832120006D8133614361536FF
:1062F0001636173612000E360F3610361136123695
:106300001200173216321532143213321200F9DF2E
:106310001232113210320F320E32120018AE04D087
:1063200019681A681B681C68120019AE03D01A6835
:106330001B681C6812001AAE02D01B681C68120091
:106340001BAE01D01C6812003B923ABE3B828CDE31
:10635000280E0B6ED8906EEC31F088EC31F003D83B
:106360000B2EF8D7120077EC3BF00A0E0A6E00EE07
:106370000EF0EF50E8B6FD0FE8BED00FEE6E0A2E1D
:10638000F8D784EC3BF012003FD812AE09D0132AA4
:10639000D8B4142AD8B4152AD8B4162AD8B4172ACF
:1063A0003BEC30F035D030D812AE09D0132AD8B437
:1063B000142AD8B4152AD8B4162AD8B4172A13C068
:1063C0000EF014C00FF015C010F016C011F017C079
:1063D00012F03ABE7CEC38F0120016D813C00EF062
:1063E00014C00FF015C010F016C011F017C012F055
:1063F0003ABE7CEC38F0120007D835EC30F008D00B
:1064000003D83BEC30F004D017EC34F00CEF32F052
:10641000C9EC32F02DEF34F04CD803E134EC30F01D
:106420001AD01AD87F0E226E2250265E2350275A89
:1064300026C00AF026520FE026BE06D0D89074EC93
:1064400031F00A2EFBD707D00A1E0A2AD89087EC13
:1064500031F00A2EFBD712003A9E2CBE3A8E2C9EAB
:1064600034EC30F028C00FF029C010F02AC011F031
:106470002BC012F02CC013F0D89074EC31F088ECE3
:1064800031F0128E13C026F0136AD89074EC31F0FC
:106490001200040E0A6EEE6608D00A2EFCD7EECF6C
:1064A000E8FF7F0B03E1D88401D0D89484EC3BF063
:1064B000120077EC3BF000EE28F0EBD777EC3BF0E6
:1064C00000EE2DF0E6D777EC3BF000EE32F0E1D7AE
:1064D00077EC3BF000EE18F0DCD777EC3BF000EE09
:1064E0001DF0D7D777EC3BF000EE0EF00A0E0A6EE7
:1064F000EE66DBD70A2EFCD7D6D71C6A1BBE1C68FB
:1065000035D01B6A1C6A1AAE31D01B681C682ED0AD
:106510001A6A1B6A1C6A19AE29D01A681B681C68A3
:1065200025D0196A1A6A1B6A1C6A18AE1FD019682E
:106530001A681B681C681AD034EC30F03A9E1C6A4A
:106540001DD034EC30F03A9E1B6A1C6A17D034EC34
:1065500030F03A9E1A6A1B6A1C6A10D034EC30F094
:106560003A9E196A1A6A1B6A1C6A08D034EC30F029
:106570003A9E1CAE03D08BEC38F03A8E18C013F064
:1065800019C014F01AC015F01BC016F01CC017F08B
:1065900000D07F0E266E000E276E72EC32F006E100
:1065A000286A296A2A6A2B6A2C6A36D033EC33F0BF
:1065B00007E0D89087EC31F0262AD8B4272AF6D7FE
:1065C00013B00AD0D89074EC31F026062628D8B43F
:1065D0002706D8B42652F4D70FA00BD00F800F2A6D
:1065E000D8B4102AD8B4112AD8B4122AD8B4132A8D
:1065F000DDD70E6A139026C013F087EC31F00FC080
:1066000028F010C029F011C02AF012C02BF013C0DE
:106610002CF02C9E3ABE2C8E1200286A296A2A6A17
:106620002C6A800E2B6EF5D7286829682A687F0EA1
:106630002B6E7F0E2C6EEDD77F0E186E000E196E2E
:106640002750195C02E12650185CD8B003D0ECDF6B
:10665000D88401D0D894120027AE03D0DEDFD884CE
:1066600001D0D894120077EC3BF000EE17F0040E46
:106670000A6EED660AD00A2EFCD7010EEF6201D039
:1066800002D0EF6602D0D88401D0D89484EC3BF0DD
:1066900012001DC000F11EC001F11FC002F120C098
:1066A00003F121C004F193EC33F00EC007F10FC0E9
:1066B00008F110C009F111C00AF112C00BF100C1BC
:1066C00018F001C119F002C11AF003C11BF004C196
:1066D0001CF079EC33F007C113F008C114F009C1C4
:1066E00015F00AC116F00BC117F03A9E3BB23A8E74
:1066F0001200BADC280E0B6ED89005D87BEC31F076
:106700000B2EFAD7120077EC3BF0050E0A6E00EE66
:1067100018F0D890EF50E8200700EE6E0A2EFAD756
:1067200084EC3BF0120077EC3BF09EDC280E0B6E05
:10673000D8906EEC31F088EC31F000EE18F0050ED8
:106740000A6EEFAE02D0300EEF5EEFA602D0030E5F
:10675000EF5EEE520A2EF5D70B2EEAD784EC3BF013
:10676000120002D83BEF31F077EC3BF09ADD00EEFF
:106770000EF010EE1DF0040E0A6EE650EE5EE650CE
:10678000EE5A0A2EFCD784EC3BF0120002D83BEF05
:1067900031F077EC3BF085DD00EE0EF010EE1DF0F1
:1067A000E650EE26040E0A6EE650EE220A2EFCD7C4
:1067B00084EC3BF0120000C118F001C119F002C1D5
:1067C0001AF003C11BF004C11CF005C122F006C180
:1067D00023F0120007C11DF008C11EF009C11FF00F
:1067E0000AC120F00BC121F00CC124F00DC125F02D
:1067F00012000FC000F110C001F111C002F112C06F
:1068000003F113C004F126C005F127C006F1120000
:106810000FC007F110C008F111C009F112C00AF150
:1068200013C00BF126C00CF127C00DF112002DC0D2
:1068300028F02EC029F02FC02AF030C02BF031C034
:106840002CF0120032C028F033C029F034C02AF0F6
:1068500035C02BF036C02CF0120028C02DF029C016
:106860002EF02AC02FF02BC030F02CC031F01200D7
:1068700028C032F029C033F02AC034F02BC035F0E4
:106880002CC036F0120094EC3BF016E291EC3BF099
:1068900013E25EEC32F01AE063EC32F017E0A9ECA0
:1068A0003BF004E35EEC32F001E306D0ACEC3BF0ED
:1068B00006E363EC32F003E3D1EC3BF01200A9EC09
:1068C0003BF003E3C6EC3BF003D00DD04EEC30F0D0
:1068D00031BE03D036AE01D0318E31AE03D036BEDC
:1068E00001D0318E12001DD83A9E3ABA3A7E3ABC97
:1068F0003A7E38EC38F012C000F113C001F114C038
:1069000002F115C003F116C004F11ED8C9EC33F032
:106910003BEC31F048EC30F07F0E1D6EB4EC33F000
:106920001ED03A9A3A9C31BE3A8A36BE3A8C7FDF04
:106930002CEC32F05EDF86DF2CEC32F069DF33ECDA
:1069400030F039DFEAEF33F033EC30F022C018F0EA
:1069500023C019F024C01DF025C01EF012000EC087
:1069600026F00FC027F034EC30F000C10FF001C169
:1069700010F002C111F003C112F004C113F0CDEC0C
:1069800032F02DEF34F094EC3BF009E291EC3BF067
:1069900006E25EEC32F006E163EC32F019E1D1EC94
:1069A0003BF01200ACEC3BF003E3A9EC3BF0F7E268
:1069B00063EC32F010E1C6EC3BF031BE03D036AEF2
:1069C00001D0318E31AE03D036BE01D0318E1200EF
:1069D000DBEC3BF0F2D7A5DF3A9E3ABA3A7E3ABCFE
:1069E0003A7E06EC39F005DFAFDFB4EC33F03BEC78
:1069F00031F048EC30F07F0E1D6EC9EC33F0AFD7AC
:106A000063EC32F001E11200367E00D094EC3BF0F2
:106A100004E291EC3BF001E203D0D1EC3BF0120038
:106A200063EC32F001E112005EEC32F003E16AEC5B
:106A300030F0120017D8C9EC33F022C026F023C082
:106A400027F03A9E12AE03D03A8E7CEC38F00EC09E
:106A500000F10FC001F110C002F111C003F112C02A
:106A600004F181D75EDFFE0E266E000E276E2550E4
:106A7000235C02E12450225C27E013E3242AD8B4EB
:106A8000252A2750255C02E12650245C07E148ECCA
:106A900030F022C024F023C025F016D0D89018DCA6
:106AA000E6D7222AD8B4232A2750235C02E12650B5
:106AB000225C07E141EC30F024C022F025C023F035
:106AC00003D0D8900BDCD3D73ABA8BEC38F03ABC71
:106AD0009AEC38F0120075EC30F043EF34F05EECD5
:106AE00032F02DE031BE2CD094EC3BF028E280EC6B
:106AF00030F0ECD848DF04EC31F01E0E0D6E0D4E78
:106B00001ED05FEC30F096EC30F03DDF96EC30F0CC
:106B10007DDFDCD838DF96EC30F03650315C0BE1AD
:106B20003550305C08E134502F5C05E133502E5C69
:106B300002E132502D5C03E004EC31F0E0D71200AA
:106B4000D1EC3BF012005EEC32F008E13F0E316E0A
:106B5000800E306E2D6A2E6A2F6A120001013F0EE0
:106B6000266F800E256F226B236B246B3F0E216FE7
:106B7000800E206F1D6B1E6B1F6B00010FEC31F040
:106B800004EC31F022C10EF123C10FF124C110F148
:106B900025C111F126C112F11E0E0D6E8BEC30F0E5
:106BA000C2EC30F0F0DE54EC30F006EC35F054EC92
:106BB00030F03650315C0BE13550305C08E1345038
:106BC0002F5C05E133502E5C02E132502D5C17E062
:106BD0000D4E15D080EC30F0CDEC30F06FD816DFD4
:106BE00025EC31F0C2EC30F04EDE1AEC31F0A1ECC5
:106BF00030F096EC30F047DE04EC31F0CFD71200E5
:106C00005EEC32F008E13F0E316E800E306E2D6A80
:106C10002E6A2F6A12002DC02CF12EC02DF12FC02C
:106C20002EF130C02FF131C030F1FCEC31F03BD807
:106C30002ADE89DF30EC31F02CC12DF02DC12EF091
:106C40002EC12FF02FC130F030C131F004EC32F002
:106C50003A943ABE3A8413C00DF027C12DF028C1F2
:106C60002EF029C12FF02AC130F02BC131F00D5286
:106C700006E03AA4C5D83AB4D5D80D2EFAD71200FA
:106C8000420E366E480E356E326A336A346A12002E
:106C9000400E366E490E356E0F0E346EDA0E336EC0
:106CA000A20E326E1200400E366E130E356E5D0E61
:106CB000346E8D0E336EDE0E326E12003F0E366E67
:106CC000800E356E326A336A346A1200400E366EB8
:106CD000326A336A346A356A1200410E366E200E0B
:106CE000356E326A336A346A1200420E366EC80E4E
:106CF000356E326A336A346A1200440E366E7A0E8A
:106D0000356E326A336A346A1200460E366E1C0ED5
:106D1000356E400E346E326A336A1200470E366E9C
:106D2000C30E356E500E346E326A336A1200490E4D
:106D3000366E740E356E240E346E326A336A12006B
:106D40004B0E366E180E356E960E346E800E336E08
:106D5000326A12004C0E366EBE0E356EBC0E346EAC
:106D6000200E336E326A12004E0E366E6E0E356E87
:106D70006B0E346E280E336E326A12003D0E366E84
:106D8000CC0E356ECC0E346ECC0E336ECD0E326E14
:106D900012003C0E366E230E356ED70E346E0A0E80
:106DA000336E3D0E326E12003A0E366E830E356E25
:106DB000120E346E6E0E336E980E326E1200350E59
:106DC000366E860E356E370E346EBD0E336E060E81
:106DD000326E1200300E366E890E356E700E346EC5
:106DE0005F0E336E410E326E12002B0E366E8C0E1D
:106DF000356EBC0E346ECC0E336E090E326E120040
:106E00006CDF43EF34F071DF43EF34F076DF43EFB4
:106E100034F07BDF43EF34F081DF43EF34F087DF82
:106E200043EF34F05ADFC3EF34F05FDFC3EF34F0E9
:106E300064DFC3EF34F069DFC3EF34F06FDFC3EF1B
:106E400034F075DFC3EF34F05EEC32F003E1D1ECE7
:106E50003BF0120080EC30F001013F0E176F800E06
:106E6000166F136B146B156B000128DF00EC35F007
:106E70000FEC31F05FEC30F021DF06EC35F01AEC6E
:106E800031F0A1EC30F0C2EC30F0C3EC34F00FEC98
:106E900031F025EC31F080EC30F0280E0D6E8BECEB
:106EA00030F014DF06EC35F004EC31F0A1EC30F0FA
:106EB000D8EC30F043EC34F0D8EC30F043EC34F064
:106EC0000FEC31F096EC30F0C3EC34F054EC30F0D1
:106ED00006EC35F054EC30F03650315C0BE13550B7
:106EE000305C08E134502F5C05E133502E5C02E148
:106EF00032502D5C05E00D4E03D080EC30F0CFD742
:106F0000E5DE43EF34F00101276B00016DEC36F054
:106F100048D806E312EC37F00101272B0001F6D721
:106F200093DFC1DEC3EC34F033EC30F027C113F053
:106F3000135206E0C9EC32F038EC34F006EC35F0D0
:106F400012007ED81CAE14D021AE29D05AD81C50C5
:106F5000215C0BE11B50205C08E11A501F5C05E12D
:106F600019501E5C02E118501D5CD8B016D017D025
:106F70001CBE02D021BE11D044D81C50215C0BE1B4
:106F80001B50205C08E11A501F5C05E119501E5C83
:106F900002E118501D5CD8B002D0D89001D0D88042
:106FA00012004ED81CAE14D021AE29D02AD81C50C5
:106FB000215C0BE11B50205C08E11A501F5C05E1CD
:106FC00019501E5C02E118501D5CD8B016D017D0C5
:106FD0001CBE02D021BE11D014D81C50215C0BE184
:106FE0001B50205C08E11A501F5C05E119501E5C23
:106FF00002E118501D5CD8B002D0D88001D0D890E2
:1070000012005EEC32F003E141EC30F00FD0D8908A
:1070100062EC31F0D8901B321A32193218321B8EC2
:1070200063EC32F003E148EC30F009D0D8905CEC2E
:1070300031F0D89020321F321E321D32208E1200C5
:107040002DC018F02EC019F02FC01AF030C01BF060
:1070500031C01CF032C01DF033C01EF034C01FF030
:1070600035C020F036C021F0120002D83BEF31F0DD
:1070700077EC3BF037D8050E0A6E00EE1DF020EEDF
:107080000EF034EC30F010EE18F0050E0B6E0AC066
:107090000CF00B500C260C060C06EF50E602F350D9
:1070A000DE26D9CF37F0DACF38F0F450DE22E86AA6
:1070B000DE220C2EFCD737C0D9FF38C0DAFF0B2EEA
:1070C000E6D7EE5220EE0EF0060E0C6E0A500C5E65
:1070D000DE520C2EFDD70A2ED6D784EC3BF03AB206
:1070E0000BD812003A921CAE02D015D83A7221AEDB
:1070F00002D020D83A7212000E1E0F1E101E111E52
:10710000121E0E2AD8B40F2AD8B4102AD8B4112AC5
:10711000D8B4122A1200181E191E1A1E1B1E1C1E7D
:10712000182AD8B4192AD8B41A2AD8B41B2AD8B421
:107130001C2A12001D1E1E1E1F1E201E211E1D2A7F
:10714000D8B41E2AD8B41F2AD8B4202AD8B4212AE9
:107150001200C8DF77EC3BF034EC30F0050E0A6E1D
:1071600000EE1DF0EE6605D00A2EFCD784EC3BF055
:1071700012000A6A0A2AD89021BE1CD01D361E367B
:107180001F362036213621501C5C0BE120501B5C41
:1071900008E11F501A5C05E11E50195C02E11D5008
:1071A000185CE8E234EC30F0D890213220321F3203
:1071B0001E321D3221501C5C0BE120501B5C08E18B
:1071C0001F501A5C05E11E50195C02E11D50185C4D
:1071D0000AE31D50185E1E50195A1F501A5A2050AB
:1071E0001B5A21501C5A7BEC31F00A2EDDD777DF79
:1071F00018C01DF019C01EF01AC01FF01BC020F0EF
:107200001CC021F03BEC31F084EF3BF0290E0A6EFC
:1072100034EC30F021501C5C0BE120501B5C08E189
:107220001F501A5C05E11E50195C02E11D50185CEC
:107230000BE31D50185E1E50195A1F501A5A205049
:107240001B5A21501C5AD88074EC31F0D89062EC53
:1072500031F021501C5C0BE120501B5C08E11F50F9
:107260001A5C05E11E50195C02E11D50185C0BE32D
:107270001D50185E1E50195A1F501A5A20501B5A82
:1072800021501C5AD8800A2EDFD7120077EC3BF031
:107290003A921CAE02D03FDF3A8234EC30F0280E36
:1072A0000A6E0A0E0B6E00EE0EF0EF500F0B0C6E16
:1072B000050E0C5CD8A002D0030EEF26EF50F00BA9
:1072C0000C6E500E0C5CD8A002D0300EEF26EC52A3
:1072D0000B2EEBD7D89062EC31F074EC31F00A2E23
:1072E000E0D784EC3BF0120094EC3BF015E2ACEC00
:1072F0003BF01CE22FD844D85AD83B941200030E1E
:10730000376409D03866372A3AB4372A030E375E15
:107310003750ABEC21F01200F2DF000EF86E600E79
:10732000F76E220EF66EBCEC21F01200E8DF000EC4
:10733000F86E600EF76E260EF66EBCEC21F01200B1
:1073400094EC3BF0E9E2ACEC3BF0F0E203D82FD850
:107350003B94120077EC3BF000EE17F011EE31F0A9
:107360000A0E0C6EEDCF0AF00A380B6E56D80AC022
:107370000BF053D80C2EF6D7E76A84EC3BF01200E2
:1073800077EC3BF0385210E001EE44F011EE44F09F
:10739000140E0A6E38C00BF0E5500A060B2EFCD70F
:1073A000E5CFEDFF0A2EFCD784EC3BF0120077EC22
:1073B0003BF00A0E0B6E38500B2637500B5CD8B0E2
:1073C00002D00BC037F03750385CD8A003D038C09B
:1073D00037F0372A3850375E3706090E0A6E3750B5
:1073E0000A5E01EE31F00A5204E0EECFE8FF0A2E09
:1073F000FCD73AA405D02B0E3ABE2D0E4CEC3AF039
:107400003A8019D83A9013D8385204E02C0E4CEC3C
:107410003AF009D884EC3BF012000B500F0B300906
:10742000E8CFE6FF120038C00CF03B9606D0010E04
:107430000C6E3B9602D037C00CF00C5226E03AA0FE
:1074400006D0EFCF0AF0300E0A5CD8A43A903BA6E3
:1074500011D00CC018F0020E186202D046EC3AF0BF
:10746000050E186202D046EC3AF0080E186202D0FF
:1074700046EC3AF0EECFE8FF3AB003D04CEC3AF0ED
:1074800002D048EC3AF00C2EDAD71200200E04D0CD
:10749000200E3BB4300E00D0DBEC20F0120077EC75
:1074A0003BF00A0E0A6E38500A5E00EE0EF0EF5006
:1074B0000A4E0CD0EF500A4E02D0EE52F8D7EE52E0
:1074C000186E490E186409D0010E06D00F0B186E05
:1074D000040E186402D0100EEF260A0E0A6E00EE9B
:1074E0000EF0EF500700EE6EE86AEF220A2EF9D791
:1074F00084EC3BF0120077EC3BF0050E0A6E0A0EAE
:107500000B6E00EE17F0EDCF18F01850F00B07E1FE
:107510000B0618500F0B03E10B060A2EF4D70BC015
:1075200018F00B5084EC3BF01200DBEC3BF034EC39
:1075300030F046EC39F00EC013F00FC014F010C05C
:1075400015F011C016F012C017F0050E376E386A2C
:107550003A943B943A983B96120094EC3BF044E208
:10756000ACEC3BF041E217EC34F00CEC32F00EC026
:1075700000F10FC001F110C002F111C003F112C0FF
:1075800004F113C018F014C019F015C01AF016C099
:107590001BF017C01CF046EC39F00EC007F10FC00D
:1075A00008F110C009F111C00AF112C00BF100C1BD
:1075B00018F001C119F002C11AF003C11BF004C197
:1075C0001CF0A4EC31F007C113F008C114F009C19C
:1075D00015F00AC116F00BC117F0140E376E0A0E23
:1075E000386E3A983B963B943A94120080EC30F017
:1075F000396A319E5EEC32F014E06DEC36F0D1EC7D
:1076000037F001E004E312EC37F0392AF6D75EECEC
:1076100036F0A1EC37F005E004E300EC37F0390672
:10762000F6D7ADEC3AF05FEC30F031BE3A8E0B0E8F
:10763000376E0A0E386E3A843A981200A0EC39F090
:10764000650E4CEC3AF03A9E39BE3A8E39BE396C32
:1076500041EC30F039C018F095EC3AF03A844BDF49
:1076600018C037F0A0EC39F012008BEC30F054EC7D
:1076700030F000EC35F030EC31F0B7EC30F0ACEC41
:1076800030F000EC35F075EC30F027C12DF028C15A
:107690002EF029C12FF02AC130F02BC131F0C3ECFC
:1076A00034F030EC31F0CDEC30F0ACEC30F000ECFC
:1076B00035F0EEEC30F043EC34F054EC30F006EC06
:1076C00035F0120077EC3BF041EC30F0050E0A6E1D
:1076D00010EE0EF020EE18F0E6500F0BDF6EE638DD
:1076E000F00BDE120A2EF8D784EC3BF01200E9CF43
:1076F00045F1EACF46F1E1CF47F1E2CF48F1D9CFEA
:1077000049F1DACF4AF1120045C1E9FF46C1EAFF6B
:1077100047C1E1FF48C1E2FF49C1D9FF4AC1DAFFD1
:10772000120022EC34F003D017EC34F000D02C9E81
:107730007F0E2C620CD0800E2B6207D02A6605D0FB
:10774000296603D0286601D002D0D88001D0D89015
:10775000120022EC34F003D017EC34F000D02C9E51
:107760007F0E2C620BD0800E2B6208D02A6606D0CA
:10777000296604D0286602D0D88001D0D8901200A3
:1077800002D82DEF34F005D82C8E120002D82DEF40
:1077900034F07F0E2C6E800E2B6E286A296A2A6ABE
:1077A000120002D82DEF34F07F0E2C6E2868296865
:1077B0002A682B68120002D82DEF34F0286A296A53
:1077C0002A6A2B6A2C6A1200410E366EA00E356EA4
:1077D000326A336A346A1200E4EC3BF0C3EC34F0F2
:1077E00000EC36F080EC30F05EEC36F006EC35F074
:1077F00004EC31F05FEC30F05EEC36F000EC35F08C
:1078000075EC30F08BEC30F0C3EC34F012004BC16F
:107810002DF04CC12EF04DC12FF04EC130F04FC1B4
:1078200031F012EC37F000EC36F02DC055F12EC0DF
:1078300056F12FC057F130C058F131C059F1120044
:1078400055C12DF056C12EF057C12FF058C130F060
:1078500059C131F018EC37F040EC36F043EC34F01D
:107860006FEC35F02DC060F12EC061F12FC062F1D8
:1078700030C063F131C064F1120060C12DF061C10C
:107880002EF062C12FF063C130F064C131F001010C
:10789000010E656F0001DFEC36F0A1EC37F009E373
:1078A0000101040E656F00010FEC37F006EC37F0B4
:1078B00018D0D4EC36F0A1EC37F007E30101030E49
:1078C000656F00010FEC37F00CD05EEC36F0A1ECE8
:1078D00037F007E30101020E656F000106EC37F097
:1078E00000D02DC05BF12EC05CF12FC05DF130C027
:1078F0005EF131C05FF1120055C12DF056C12EF07E
:1079000057C12FF058C130F059C131F00101030EB9
:107910005A6F0001F5EC36F0A1EC37F00BE30FECF9
:1079200037F00FEC37F006EC37F00101080E5A6F14
:1079300000014CD0EAEC36F0A1EC37F009E30FEC93
:1079400037F00FEC37F00101070E5A6F00013ED0FF
:10795000DFEC36F0A1EC37F009E30FEC37F006EC82
:1079600037F00101060E5A6F000130D0D4EC36F02A
:10797000A1EC37F007E30FEC37F00101050E5A6F69
:10798000000124D05EEC36F0A1EC37F007E306EC02
:1079900037F00101040E5A6F000118D097EC36F051
:1079A000D1EC37F007E321EC37F00101010E5A6FFB
:1079B00000010CD07DEC36F0D1EC37F007E318EC89
:1079C00037F00101020E5A6F000100D02DC050F1B6
:1079D0002EC051F12FC052F130C053F131C054F1DB
:1079E000120050C12DF051C12EF052C12FF053C1E1
:1079F00030F054C131F0ADEC3AF0050E376E010EA7
:107A0000386E6DEC36F0A1EC37F003E3040E386EFF
:107A10000FD075EC36F0A1EC37F003E3030E386EAF
:107A200007D07DEC36F0A1EC37F002E3020E386EA1
:107A300067D84FEC3AF0A0EC39F05AC118F0030EB9
:107A4000186209D0000EF86E600EF76E2A0EF66E00
:107A5000BCEC21F054D0040E186209D0000EF86E70
:107A6000600EF76E2E0EF66EBCEC21F048D0050EBF
:107A7000186209D0000EF86E600EF76E320EF66EC8
:107A8000BCEC21F03CD0060E186209D0000EF86E56
:107A9000600EF76E360EF66EBCEC21F030D0070E9D
:107AA000186209D0000EF86E600EF76E3A0EF66E90
:107AB000BCEC21F024D0020E186209D0000EF86E42
:107AC000600EF76E420EF66EBCEC21F018D0010E7F
:107AD000186209D0000EF86E600EF76E460EF66E54
:107AE000BCEC21F00CD0080E186209D0000EF86E24
:107AF000600EF76E3E0EF66EBCEC21F000D0120068
:107B00007BEC3AF0030E186402D0010E386E030EBF
:107B1000186202D0020E386E020E186202D0030EF6
:107B2000386E010E186202D0040E386E000E186214
:107B300002D0040E386E12005BC12DF05CC12EF035
:107B40005DC12FF05EC130F05FC131F0ADEC3AF0B5
:107B5000060E376E010E386E7DEC36F0A1EC37F074
:107B600002E3020E386E75EC36F0A1EC37F002E35A
:107B7000030E386E6DEC36F0A1EC37F002E3040E24
:107B8000386EBEDF4FEC3AF0A0EC39F065C118F06A
:107B9000010E186209D0000EF86E600EF76E4A0EE4
:107BA000F66EBCEC21F024D0020E186209D0000E53
:107BB000F86E600EF76E4E0EF66EBCEC21F018D02B
:107BC000030E186209D0000EF86E600EF76E520EAA
:107BD000F66EBCEC21F00CD0040E186209D0000E39
:107BE000F86E600EF76E560EF66EBCEC21F000D00B
:107BF00012004BC12DF04CC12EF04DC12FF04EC1E3
:107C000030F04FC131F0ADEC3AF0050E376E020E98
:107C1000386E4FEC3AF07BEC3AF0030E186004D06B
:107C2000040E376E020E386E020E186404D0040E75
:107C3000376E010E386E24D04BC12DF04CC12EF0A2
:107C40004DC12FF04EC130F04FC131F0ADEC3AF0E4
:107C5000040E376E010E386E4FEC3AF07BEC3AF0C2
:107C6000030E186004D0030E376E010E386E020E3C
:107C7000186406D0040E376E000E386E4FEC3AF0E2
:107C80003A84A0EC39F0000EF86E600EF76E5A0ED2
:107C9000F66EBCEC21F0120050C12DF051C12EF057
:107CA00052C12FF053C130F054C131F0ADEC3AF075
:107CB000040E376E010E386E6DEC36F0A1EC37F025
:107CC00003E3030E386E0FD075EC36F0A1EC37F0FD
:107CD00003E3020E386E07D07DEC36F0A1EC37F0EE
:107CE00002E3010E386E4FEC3AF065D8A0EC39F0A3
:107CF0005AC118F0030E186209D0000EF86E600E1B
:107D0000F76E2A0EF66EBCEC21F054D0040E186209
:107D100009D0000EF86E600EF76E2E0EF66EBCECFB
:107D200021F048D0050E186209D0000EF86E600EE2
:107D3000F76E320EF66EBCEC21F03CD0060E1862E7
:107D400009D0000EF86E600EF76E360EF66EBCECC3
:107D500021F030D0070E186209D0000EF86E600EC8
:107D6000F76E3A0EF66EBCEC21F024D0020E1862CB
:107D700009D0000EF86E600EF76E420EF66EBCEC87
:107D800021F018D0010E186209D0000EF86E600EB6
:107D9000F76E460EF66EBCEC21F00CD0080E1862A1
:107DA00009D0000EF86E600EF76E3E0EF66EBCEC5B
:107DB00021F000D012007BEC3AF0030E186404D0DE
:107DC000050E376E000E386E030E186202D0010EDB
:107DD000386E020E186202D0020E386E010E186262
:107DE00002D0030E386E000E186202D0030E386EF9
:107DF000120050C12DF051C12EF052C12FF053C1CD
:107E000030F054C131F0ADEC3AF0030E376E010E94
:107E1000386E6DEC36F0A1EC37F003E3020E386EED
:107E200011D075EC36F0A1EC37F003E3010E386E9B
:107E300009D07DEC36F0A1EC37F004E3000E386E8B
:107E4000040E376E4FEC3AF065D8A0EC39F05AC109
:107E500018F0030E186209D0000EF86E600EF76E6F
:107E60002A0EF66EBCEC21F054D0040E186209D034
:107E7000000EF86E600EF76E2E0EF66EBCEC21F062
:107E800048D0050E186209D0000EF86E600EF76E2D
:107E9000320EF66EBCEC21F03CD0060E186209D012
:107EA000000EF86E600EF76E360EF66EBCEC21F02A
:107EB00030D0070E186209D0000EF86E600EF76E13
:107EC0003A0EF66EBCEC21F024D0020E186209D0F6
:107ED000000EF86E600EF76E420EF66EBCEC21F0EE
:107EE00018D0010E186209D0000EF86E600EF76E01
:107EF000460EF66EBCEC21F00CD0080E186209D0CC
:107F0000000EF86E600EF76E3E0EF66EBCEC21F0C1
:107F100000D012007BEC3AF0030E186404D0040E7B
:107F2000376E000E386E030E186204D0040E376EE2
:107F3000000E386E020E186202D0010E386E010E6D
:107F4000186202D0020E386E000E186202D0020EC5
:047F5000386E120075
:020000040030CA
:0300010028192398
:02000500BD80BC
:0200000400F00A
:10000000812602F94102812602F941010000010026
:10001000050200000020420000002042986E12837A
:100020003C00000086C2986E12833C00000086C22D
:10003000986E12833C00000086C2986E12833C00CA
:10004000000086C2C800FA2C307532001E1E0E0059
:00000001FF
